:020000040800F2
:1000000000070020F1010008D52B00088D2B000807
:10001000B52B00088D2B0008AD2B0008F30100085C
:10002000F3010008F3010008F3010008C93B0008D0
:10003000F3010008F3010008F3010008F3010008D0
:10004000F3010008F3010008F3010008F3010008C0
:10005000F3010008F30100085D61000885610008F4
:10006000AD610008D5610008FD610008F3010008DA
:10007000F3010008F3010008F3010008F301000890
:10008000F3010008F3010008F3010008412B000808
:100090006D2B00087D2B0008F30100082562000885
:1000A000F3010008F3010008F3010008F301000860
:1000B000F9620008F3010008F3010008F3010008E9
:1000C000F3010008F3010008F3010008F301000840
:1000D000F3010008F3010008F3010008F301000830
:1000E00089620008F3010008F3010008F301000829
:1000F000F3010008F3010008F3010008F301000810
:10010000F3010008F3010008F3010008F3010008FF
:10011000F3010008F3010008F3010008F3010008EF
:10012000F3010008F3010008F3010008F3010008DF
:10013000F3010008F3010008F3010008F3010008CF
:10014000F3010008F3010008F3010008515700080B
:10015000F3010008F3010008F3010008F3010008AF
:10016000F3010008F3010008F3010008F30100089F
:10017000F3010008F3010008F3010008F30100088F
:10018000F3010008F3010008F3010008F30100087F
:10019000F3010008F3010008F3010008F30100086F
:1001A000F3010008F3010008F3010008F30100085F
:1001B000F3010008F3010008F3010008F30100084F
:1001C000F3010008F3010008F3010008F30100083F
:1001D000F3010008F3010008F3010008F30100082F
:1001E0006915000800000000000000000000000089
:1001F00002E000F000F8FEE772B6374880F30888A6
:10020000364880F3098836483649086040F20000D5
:10021000CCF200004EF63471CEF200010860BFF35C
:100220004F8FBFF36F8F40F20000C0F2F0004EF628
:100230008851CEF200010860BFF34F8FBFF36F8F7C
:100240004FF00000E1EE100A4EF63C71CEF20001D4
:100250000860062080F31488BFF36F8F04F040FF1E
:1002600005F024FE4FF055301F491B4A91423CBF18
:1002700041F8040BFAE71D49184A91423CBF41F886
:10028000040BFAE71A491B4A1B4B9A423EBF51F82E
:10029000040B42F8040BF8E700201849184A914271
:1002A0003CBF41F8040BFAE704F01EFF05F052FED4
:1002B000144C154DAC4203DA54F8041B8847F9E797
:1002C00000F042F8114C124DAC4203DA54F8041B12
:1002D0008847F9E704F006BF00070020002300204C
:1002E0000000000808ED00E00001002000070020E9
:1002F000E068000800230020B0230020B023002085
:1003000044560020E0010008E4010008E401000870
:10031000E40100082DE9F04F2DED108AC1F80CD052
:10032000C3689D46BDEC108ABDE8F08F002383F3BF
:1003300011882846A047002004F0D8F9FEE704F011
:1003400057F900DFFEE70000F8B501F073F904F09B
:1003500061FE074604F0B0FE0546A8BB1F4B9F4256
:1003600032D001339F4232D01D4B27F0FF029A4218
:1003700030D1F8B200F016FF2E4642F2107400F0B1
:1003800017FF08B10024264601F000FD20B103202C
:1003900000F07AF80024264635B1124B9F4203D074
:1003A00004F082FE00242646002004F03DFE0EB13B
:1003B00000F080F801F09AFA00F066FF204600F0A5
:1003C000DFF800F077F8F9E72E460024D7E7044677
:1003D0000126D4E7064641F28834D0E7010007B091
:1003E000000008B0263A09B008B501F0F5F8A0F110
:1003F00020035842584108BD07B541F212030221BB
:1004000001A8ADF8043001F005F903B05DF804FB74
:1004100038B5302383F31188174803680BB104F013
:1004200031FA164A144800234FF47A7104F020FA86
:10043000002383F31188124C236813B12368013B16
:100440002360636813B16368013B63600D4D2B78D3
:1004500033B963687BB9022001F0B2F932236360DB
:100460002B78032B07D163682BB9022001F0A8F980
:100470004FF47A73636038BDB02300201104000884
:10048000D0240020C8230020084B187003280CD863
:10049000DFE800F008050208022001F087B9022019
:1004A00001F07AB9024B00225A607047C82300203D
:1004B000D024002010B501F069FC30B1294B032293
:1004C0001A70294B00225A6010BD284B284A1C463E
:1004D00019680131F8D004339342F9D16268254B91
:1004E0009A42F1D9244B9B6803F1006303F58033F2
:1004F0009A42E9D204F0ACFD04F0BEFD002001F008
:10050000B3F80220FFF7C0FF1C4B1A6C00221A64DC
:10051000196E1A66196E596C5A64596E5A665A6E7B
:100520005A6942F080025A615A6922F080025A6187
:100530005A691A6942F000521A611A6922F000528F
:100540001A611B6972B64FF0E0233021C3F8084DE1
:10055000D4E9003281F311889D4683F3088810475F
:10056000B2E700BFC8230020D0240020000001080B
:1005700020000108FFFF000800230020003802408F
:100580002DE9F04F93B0AC4B00902022FF210AA838
:100590009D6801F055F9A94A1378A3B9A84801212B
:1005A00003601170302383F3118803680BB104F0EA
:1005B00069F9A44AA24800234FF47A7104F058F96B
:1005C000002383F31188009B13B19F4B009A1A609C
:1005D0009E4A009C1378032B1EBF002313709A4A77
:1005E0004FF0000A18BF5360D3465646D14601204B
:1005F00001F0DCF824B1944B1B68002B00F015824D
:10060000002000F0E9FF0390039B002B01DA00F0CB
:1006100083FE039B002BEDDB012001F0BDF8039B63
:10062000213B162BE3D801A252F823F089060008DB
:10063000B106000845070008EF050008EF050008AF
:10064000EF050008CF0700089F090008B908000857
:100650001B0900084309000869090008EF050008A4
:100660007B090008EF050008ED09000829070008CC
:10067000EF050008310A0008950600082907000860
:10068000EF0500081B0900080220FFF7ADFE002857
:1006900040F0F581009B0221BAF1000F08BF1C4613
:1006A00005A841F21233ADF8143000F0B3FF9EE715
:1006B0004FF47A7000F090FF071EEBDB0220FFF78B
:1006C00093FE0028E6D0013F052F00F2DA81DFE833
:1006D00007F0030A0D10133605230593042105A81E
:1006E00000F098FF17E054480421F9E75848042126
:1006F000F6E758480421F3E74FF01C08404600F0A5
:10070000B5FF08F104080590042105A800F082FF58
:10071000B8F12C0FF2D1012000FA07F747EA0B0BD2
:100720005FFA8BFB4FF0000901F0D6F826B10BF011
:100730000B030B2B08BF0024FFF75EFE57E746486C
:100740000421CDE7002EA5D00BF00B030B2BA1D17C
:100750000220FFF749FE074600289BD0012000F049
:1007600083FF0220FFF790FE00261FFA86F840461E
:1007700000F08AFF044690B10021404600F09CFF43
:1007800001360028F1D1BA46044641F21213022183
:1007900005A8ADF814303E4600F03CFF27E70120E5
:1007A000FFF772FE2546244B9B68AB4207D92846CB
:1007B00000F05CFF013040F067810435F3E7234B24
:1007C00000251D70204BBA465D603E46ACE7002E0A
:1007D0003FF460AF0BF00B030B2B7FF45BAF0220F9
:1007E000FFF752FE322000F0F7FEB0F10008FFF6EE
:1007F00051AF18F003077FF44DAF0F4A926808EB32
:10080000050393423FF646AFB8F5807F3FF742AF0E
:10081000124B0193B84523DD4FF47A7000F0DCFEF3
:100820000390039A002AFFF635AF019B039A03F861
:10083000012B0137EDE700BF00230020CC2400206E
:10084000B023002011040008D0240020C823002079
:1008500004230020082300200C230020CC230020A8
:10086000C820FFF7C1FD074600283FF413AF1F2D36
:1008700011D8C5F1200242450AAB25F0030028BF7C
:10088000424683490192184400F0B4FF019A80481F
:10089000FF2100F0D5FF4FEAA8037D490193C8F37B
:1008A0008702284600F0D4FF064600283FF46DAFCB
:1008B000019B05EB830537E70220FFF795FD002834
:1008C0003FF4E8AE00F018FF00283FF4E3AE002745
:1008D000B846704B9B68BB4218D91F2F11D80A9B92
:1008E00001330ED027F0030312AA134453F8203C1F
:1008F00005934046042205A901F000FA043780461A
:10090000E7E7384600F0B2FE0590F2E7CDF8148034
:10091000042105A800F07EFE06E70023642104A858
:10092000049300F06DFE00287FF4B4AE0220FFF7C0
:100930005BFD00283FF4AEAE049800F0C5FE0590C4
:10094000E6E70023642104A8049300F059FE002880
:100950007FF4A0AE0220FFF747FD00283FF49AAED7
:10096000049800F0C1FEEAE70220FFF73DFD0028F1
:100970003FF490AE00F0D0FEE1E70220FFF734FD37
:1009800000283FF487AE05A9142000F0CBFE042117
:100990000746049004A800F03DFE3946B9E732202E
:1009A00000F01AFE071EFFF675AEBB077FF472AEAD
:1009B000384A926807EB090393423FF66BAE022078
:1009C000FFF712FD00283FF465AE27F003074F4400
:1009D000B9453FF4A9AE484600F048FE0421059011
:1009E00005A800F017FE09F10409F1E74FF47A7049
:1009F000FFF7FAFC00283FF44DAE00F07DFE002822
:100A000044D00A9B01330BD008220AA9002000F031
:100A10001FFF00283AD02022FF210AA800F010FF73
:100A2000FFF7EAFC1C4803F067FE13B0BDE8F08F47
:100A3000002E3FF42FAE0BF00B030B2B7FF42AAEEE
:100A40000023642105A8059300F0DAFD074600287D
:100A50007FF420AE0220FFF7C7FC804600283FF459
:100A600019AEFFF7C9FC41F2883003F045FE059846
:100A700000F064FF464600F02FFF3C46B7E506460F
:100A800052E64FF0000905E6BA467EE637467CE6B8
:100A9000CC23002000230020A0860100094A13680F
:100AA00049F2690099B21B0C00FB01331360064B3D
:100AB000186844F2506182B2000C01FB0200186019
:100AC00080B27047182300201423002010B50021A5
:100AD0001022044600F0B4FE034B03CB206061609B
:100AE0001868A06010BD00BF107AFF1F2DE9F0410B
:100AF000ADF5507D0DF13C086EAC40F27512074625
:100B00000D4610A80021C8F8001000F099FE4FF41F
:100B1000C4720021204600F093FE02F063F8254BDA
:100B20004FF47A72B0FBF2F0186093E807000223EA
:100B300084E807000DF5ED702382FFF7C7FF4FF241
:100B400003631D49238406A805F0E6FC202384F8EE
:100B500032310DF2EB2606AB0DF1380C1A4603CA02
:100B6000624530607160134606F10806F6D14146D1
:100B70000122204600F0E4FE00230393AB7E0293A3
:100B800005F11903019380B20123CDE9048000939C
:100B9000E97E06A3D3E90023384602F0EBFB0DF50E
:100BA000507DBDE8F08100BFAFF300809E6AC42194
:100BB000818A46EED8240020286500082DE9F041FE
:100BC0002C4C237ADAB080460D465BBB27A9284619
:100BD00000F0C6FF0746002842D19DF89D60C82E50
:100BE0003ED801464FF4A662204600F029FE4FF49D
:100BF0008073C4F8F8314FF40073C4F80C334FF429
:100C00004073C4F8203432460DF19E0104F109000E
:100C100000F0F0FD26449DF89C30777223720BB9EA
:100C2000EB7E23728122002106AC27A800F008FE8B
:100C30000122214627A800F0CFFF00230393AB7EBB
:100C4000029305F1190380B201932823CDE90440F2
:100C50000093E97E05A3D3E90023404602F08AFB16
:100C60005AB0BDE8F08100BFAFF300802641727238
:100C7000DF25D7B7F8450020F0B5254E4FF48A752B
:100C800005FB0065F1B096F8D83085F8DC3000241B
:100C9000D822214685F8E8403AA800F0D1FD06F1B7
:100CA000090000F0C5FDD5F8E4308DF8F000C2B2BF
:100CB00006AF06F109010DF1F100CDE93A3400F07B
:100CC00099FD394601223AA800F0B2FF80B2CDE981
:100CD000047008230127CDE9023706F1D8030193F8
:100CE00030230093317A0B4807A3D3E9002302F0A5
:100CF00041FBA04206DD01F075FFC5F8E000384673
:100D000071B0F0BD2046FBE778F6339F93CACD8DD6
:100D1000F8450020F03400202DE9F0411D4D1E4E15
:100D20001E4F86B0284602F051FB034658B30024FC
:100D3000CDE90344ADF81440027B8DF81420996886
:100D40004068029403AA03C21B68DFF8548043F092
:100D50000043029301F048FF821941F1000300941F
:100D600002A9384601F0F0F9A04205DD284602F05C
:100D700031FB88F80040D5E798F80030072B05D8FC
:100D8000013388F8003006B0BDE8F081014802F078
:100D900021FBF8E7F034002040420F00203500200E
:100DA0002D4B002070B50D4614461E4602F03EFA4B
:100DB00050B9022E10D1012C0ED112A3D3E9002379
:100DC000C5E90023012007E0282C10D005D8012C0C
:100DD00009D0052C0FD0002070BD302CFBD10BA307
:100DE000D3E90023ECE70BA3D3E90023E8E70BA347
:100DF000D3E90023E4E70BA3D3E90023E0E700BF36
:100E0000AFF30080401DA12026812A0B78F6339F86
:100E100093CACD8D9E6AC421818A46EE26417272A4
:100E2000DF25D7B7F017304A39059E5638B5054645
:100E30000E4C0021013500F03FFCA4F82C55B4F80D
:100E40002C0500F021FC78B1B4F82C0500F02CFC46
:100E5000014648B9B4F82C0500F02EFCB4F82C3546
:100E60000133A4F82C35EAE738BD00BFF84500206F
:100E700010B50A4B0A4A1A6003F5805393F86020B4
:100E80003AB9DC6D2CB1204600F0FEFF204605F09B
:100E900083FABDE81040034800F0F6BF203500207B
:100EA000E8650008684500202DE9F04F8FB000AFDD
:100EB00005460C4602F0BAF9002849D1237E022BE0
:100EC0001BD1E38A012B18D101F08CFE0646FFF7F7
:100ED000E5FD03464FF4C870DFF8C482B3FBF0F2BF
:100EE00006F5167602FB103316FA83F3C8F80030C5
:100EF000E37E33B9A34B00221A703C37BD46BDE8F0
:100F0000F08F07F12401204600F0E8FD0028F4D11D
:100F100007F11400FFF7DAFD97F8264007F11401F6
:100F2000224607F1270005F081FA0028E2D10F2CB4
:100F300008D8944B1C70D8F80030A3F51673C8F885
:100F40000030DAE797F82410284602F067F9D4E772
:100F5000E38A282B2BD010D8012B23D0052BCCD102
:100F6000BFF34F8F8849894BCA6802F4E06213438C
:100F7000CB60BFF34F8F00BFFDE7302BBDD1844E58
:100F8000E17E327A9142B8D1607E3146002291F8FA
:100F9000DC50854200F0A5800132042A01F58A71F7
:100FA000F5D1AAE721462846FFF7A0FDA5E721468F
:100FB0002846FFF703FEA0E7B2F8EC507B6005F18E
:100FC00003094FEA99094FEA8902D11DC908A8EB24
:100FD000C1039D46EB460021584600F031FC04F168
:100FE000EE012A463144584600F004FC7B6813B9F0
:100FF000012000F039FB96F8D20000F045FB0446D2
:1010000030B9307200F078FB204600F02DFBB1E0E3
:10101000D6F8D4203AB996F8D200B6F82C258242F8
:1010200001D8FFF703FFD6F8D4202A44944208D20F
:1010300096F8D200B6F82C250130824201D8FFF78D
:10104000F5FE70685FFA89F2594600F001FC08B9B4
:10105000C54679E0726896F8D2002A447260D6F8E4
:10106000D42005EB0209C6F8D49000F00DFB8145B1
:1010700009D396F8D220D6F8D4000132001B86F8A6
:10108000D220C6F8D400FF2D0FD80024347200F00F
:1010900033FB204600F0E8FA00F078FE3D4B188163
:1010A00008B9FFF707FAC54627E7BB6896F8D900E5
:1010B0000AFB0362FB68D2F8E41082F8E83001F51D
:1010C0008061C2F8E030C2F8E410FFF7D5FDFFF709
:1010D00023FE96F8D920013202F0030286F8D920C7
:1010E000B6E74FF48A7A0AFB02F505F1EA013144CA
:1010F000204600F0C9FDF86000287FF4FEAE3544BC
:10110000012285F8E82001F06DFDD5F8E020D6ED4C
:10111000007ADFED216A801A192838BF192040F6BD
:10112000B832904228BF1046B8EE677A07EE900AB0
:10113000F8EEE77A67EEA67ADFED186AE7EE267A30
:10114000FCEEE77AC6ED007A96F8D930BB60BA6853
:1011500073680AFB02F4321992F8E81059B1D2F818
:10116000E4108B42E8463FF427AF002182F8E810F4
:10117000C2F8E010C5467368064A9B0A0133138122
:10118000BBE600BFE934002000ED00E00400FA05F2
:10119000F8450020D8240020CDCCCC3D6666663FC3
:1011A000EC340020014B1870704700BFE42400208D
:1011B00030B54FF000542B4B22689A4285B007D0CF
:1011C00003F084FF044620BB0024204605B030BD58
:1011D000254B627D25481A70237D03724FF480737E
:1011E000C0F8F8314FF40073C0F80C3300254FF409
:1011F0004073C0F820341E49C0F8E450C9220930B9
:1012000000F0F8FA2046E022294600F019FB0124FC
:10121000DBE7184A184D136C43F000731364AA6D92
:10122000164B9A42D0D12B6E013B7E2BCCD8144A60
:1012300007CA01AB83E807001846032100F074FDDC
:101240006B6D83424FF00003BED12A6D8A4201BF0D
:10125000AB65054B2A6E1A7003BF0A4BEA6D1A6024
:101260001C46B2E79AAD44C5E4240020F8450020AE
:101270001600002000380240006600405041A0B037
:10128000586600401023002037B51A4D00F07EFD4F
:1012900002236B71184B288119681848012201F04C
:1012A0003DFB00230193164B164900931648174B3C
:1012B0004FF4805201F08AFF154B197811B1124892
:1012C00001F0ACFF01F08EFC0446FFF7E7FB4FF4A2
:1012D000C873B0FBF3F202FB130304F5167010FAA7
:1012E00083F00C4B186003F0E7FE08B10F232B814D
:1012F00003B030BDD824002010230020203500206A
:10130000A50D0008E8240020F0340020A90E0008F4
:10131000E4240020EC3400202DE9F04F2DED028B69
:101320000FF23829D9E90089834C93B00BAE9FEDB9
:101330007E8BFFF7F1FC814FDFF828A200230A9390
:10134000ADF834300B9373604FF0000B5B468DEDBE
:10135000008B01250DF11D0207A938468DF81C50A0
:101360008DF81DB001F088FA9DF81C30002B40F07C
:10137000A580204601F05AFF0646002845D1704F4F
:1013800001F030FC3B6898423FD301F02BFC8246D1
:10139000FFF784FB4FF4C873B0FBF3F202FB1303B7
:1013A0000AF5167010FA83F03860664F97F800B0AF
:1013B000CBF1100ABBF1000F14BF33462B465FFA86
:1013C0008AFA0EA88DF82830FFF780FBBAF1060FD5
:1013D00028BF4FF0060A0EAB03EB0B0152460DF18E
:1013E000290000F007FA0AAB0393182302930AF1CD
:1013F0000102554BD2B2CDE90053049220464CA3D2
:10140000D3E9002301F058FF3E7001F0EBFB4F4A97
:101410004F4D1368C31AB3F57A7F2ED3106001F0D5
:10142000E3FB02460B46204601F0DEFF204601F0BA
:10143000FDFE10B32B7A474E002B14BF032302236B
:10144000737101F0CFFB0EAF4FF47A730122B0FB42
:10145000F3F039463060304600F018FB1823029351
:101460003D4B019380B240F25513CDE903700093D8
:1014700042464B46204601F01FFF2B7A93B101F004
:10148000B1FB002607464FF48A7A95F8D90030441C
:1014900000F003000AFB005393F8E82092B30136F2
:1014A000042EF2D1C82003F027F92B7A002B7FF409
:1014B0003DAF13B0BDEC028BBDE8F08FDAF814300D
:1014C00083F48043CAF81430594610220EA800F065
:1014D000B7F90DF11E0308AA0AA9384600F034FF37
:1014E00096E803000FAB83E803009DF834308DF8D5
:1014F00044300A9B0E930EA9DDE90823204602F032
:1015000047F921E7D3F8E02042B12B68FA2B38BF26
:10151000FA23BA1A0533B2EB430FC0D3FFF7ACFB83
:101520000028BCD1BEE700BF0000000000000000A2
:10153000401DA12026812A0BF034002020350020F8
:10154000EC340020E9340020E8340020284B00204F
:10155000F8450020D82400202C4B0020F1C6A7C15C
:10156000D068080F0000024008B5054800F088FF69
:10157000BDE80840034A0449002004F007BF00BF4B
:1015800020350020684B0020710E000870B50F4B0D
:101590001B780133DBB2012B0C4611D80C4D2968A6
:1015A0004FF47A730E6AA2FB0332014622462846A4
:1015B000B047844204D1074B00221A70012070BD4D
:1015C0004FF4FA7003F098F80020F8E71C2300208D
:1015D000E04D00205C4B002007B5002302460121AE
:1015E0000DF107008DF80730FFF7D0FF20B19DF80F
:1015F000070003B05DF804FB4FF0FF30F9E700008F
:101600000A4608B50421FFF7C1FF80F00100C0B20F
:10161000404208BD30B4054C2368DD69044B0A46DE
:10162000AC460146204630BC604700BFE04D00207C
:10163000A086010070B503F08FFB094E094D308084
:10164000002428683388834208D903F07FFB2B6885
:1016500004440133B4F5803F2B60F2D370BD00BF6A
:101660005E4B0020304B002003F024BC00F10060F2
:1016700000F580300068704700F10060920000F5CE
:10168000803003F0AFBB0000054B1A68054B1B8888
:101690009B1A834202D9104403F058BB00207047C4
:1016A000304B00205E4B0020024B1B68184403F0B7
:1016B00055BB00BF304B0020024B1B68184403F0A1
:1016C00065BB00BF304B002010F003030AD1B0F51A
:1016D000047F05D200F10050A0F51040D0F800388A
:1016E000184670470023FBE700F10050A0F51040BA
:1016F000D0F8100A70470000064991F8243033B141
:101700000023086A81F824300822FFF7B5BF0120C2
:10171000704700BF344B0020014B1868704700BF72
:10172000002004E070B5194B1D68194B0138C5F352
:101730000B0408442D0C04221E88A6420BD15C68C1
:101740000A46013C824213460FD214F9016F4EB192
:1017500002F8016BF6E7013A03F10803ECD181428C
:101760000B4602D22C2203F8012B0A4A05241688C4
:10177000AE4204D1984284BF967803F8016B013CD5
:1017800002F10402F3D1581A70BD00BF002004E03A
:101790008C65000878650008022802BF024B4FF0F4
:1017A00080429A61704700BF00000240022802BFD9
:1017B000024B4FF480429A61704700BF0000024024
:1017C000022801BF024A536983F480435361704782
:1017D0000000024070B504464FF47A764CB1412CBB
:1017E000254628BF412506FB05F002F085FF641B56
:1017F000F4E770BD10B50023934203D0CC5CC45411
:101800000133F9E710BD000010B5013810F9013FB0
:101810003BB191F900409C4203D11AB10131013A28
:10182000F4E71AB191F90020981A10BD1046FCE7B0
:1018300003460246D01A12F9011B0029FAD170475B
:1018400002440346934202D003F8011BFAE77047B3
:101850002DE9F8431F4D144695F824200746884685
:1018600052BBDFF870909CB395F824302BB920223E
:10187000FF2148462F62FFF7E3FF95F82400C0F1EF
:101880000802A24228BF2246D6B24146920005EB8A
:101890008000FFF7AFFF95F82430A41B1E44F6B27A
:1018A000082E17449044E4B285F82460DBD1FFF79A
:1018B00023FF0028D7D108E02B6A03EB8203834281
:1018C000CFD0FFF719FF0028CBD10020BDE8F88367
:1018D0000120FBE7344B0020024B1A78024B1A70B0
:1018E000704700BF5C4B00201C23002010B5104C3B
:1018F000104802F057FA21460E4802F07FFA246899
:10190000626DD2F8043843F00203C2F804384FF491
:101910007A70FFF75FFF0849204602F075FB626DA1
:10192000D2F8043823F00203C2F8043810BD00BF17
:10193000D4660008E04D0020DC6600087047000017
:101940002DE9F0470D46044600219046284640F216
:101950007912FFF775FF234620220021284601F067
:10196000B9FE231D02222021284601F0B3FE631D8B
:1019700003222221284601F0ADFEA31D03222521CA
:10198000284601F0A7FE04F108031022282128466A
:1019900001F0A0FE04F1100308223821284601F0CE
:1019A00099FE04F1110308224021284601F092FE1D
:1019B00004F1120308224821284601F08BFE04F1AD
:1019C000140320225021284601F084FE04F118035C
:1019D00040227021284601F07DFE04F120030822F8
:1019E000B021284601F076FE04F121030822B82137
:1019F000284601F06FFE04F12207C0263B4631461F
:101A000008222846083601F065FEB6F5A07F07F1EA
:101A10000107F3D104F1320308223146284601F0D0
:101A200059FE002704F1330A94F832304FEAC7090F
:101A30009F4209F5A47615D3B8F1000F08D13146BD
:101A400004F599730722284601F044FE09F24F1667
:101A5000274694F832213B1B93420CD3F01DC0085B
:101A6000BDE8F0870AEB070308223146284601F05B
:101A700031FE0137D8E707F23313314608222846F2
:101A800001F028FE08360137E3E7000013B50446ED
:101A90000846002101602346C0F80310202201906F
:101AA00001F018FE0198231D0222202101F012FEF0
:101AB0000198631D0322222101F00CFE0198A31D51
:101AC0000322252101F006FE019804F108031022EB
:101AD000282101F0FFFD072002B010BDF7B500235B
:101AE000047F00910E4607221946054601F0B6FC18
:101AF000731C0093012200230721284601F0AEFC4D
:101B0000C4B9B31C0093052223460821284601F0DE
:101B1000A5FC0D243746B278BB1B934211D32B7F13
:101B2000A88A0734E408BBB9844294BF002001208E
:101B300003B0F0BDAB8ADB00083BDB08B3700824C0
:101B4000E8E7FB1C0093214600230822284601F009
:101B500085FC08340137DEE7201A18BF0120E7E7CB
:101B6000F7B50023047F00910E460822194605466A
:101B700001F074FC731CC4B908220093114623467B
:101B8000284601F06BFC1024012372785F1C013B96
:101B9000934211D32B7FA88A0734E408BBB984424F
:101BA00094BF0020012003B0F0BDAB8ADB00083BEE
:101BB000DB0873700824E7E7F3190093214600233C
:101BC0000822284601F04AFC08343B46DDE7201A8B
:101BD00018BF0120E7E70000F8B50E460546144699
:101BE000002181223046FFF72BFE2B4608220021E0
:101BF000304601F06FFD7CB96B1C0722082130468E
:101C000001F068FD0F2401236A785F1C013B9342B9
:101C100004D3E01DC008F8BD0824F4E7EB19214601
:101C20000822304601F056FD08343B46ECE7000040
:101C3000F8B50E46054614460021CE223046FFF781
:101C4000FFFD2B4628220021304601F043FD7CB9E0
:101C500005F1080308222821304601F03BFD30241D
:101C60002F462A7A7B1B934204D3E01DC008F8BD9F
:101C70002824F5E707F1090321460822304601F040
:101C800029FD08340137ECE7F7B5047F00910E46D3
:101C9000012310220021054601F0E0FBC4B9B31C6A
:101CA0000093092223461021284601F0D7FB19246E
:101CB00037467288BB1B9A4211D82B7FA88A0734FB
:101CC000E408BBB9844294BF0020012003B0F0BDFA
:101CD000AB8ADB00103BDB0873801024E8E73B1D78
:101CE0000093214600230822284601F0B7FB083460
:101CF0000137DEE7201A18BF0120E7E730B5094DAC
:101D00000A4491420DD011F8013B5840082340F39A
:101D10000004013B2C4013F0FF0384EA5000F6D18D
:101D2000EFE730BD2083B8EDF7B54FF0FF33DFF8B4
:101D300054C0DFF854E000EB81011A4688421CD001
:101D400050F8044B019401AF042417F8015B82EAB8
:101D500005620825DB18164605F1FF355241002EB5
:101D6000BCBF83EA0C0382EA0E0215F0FF05F1D135
:101D7000013C14F0FF04E8D1E0E7D843D14303B0BD
:101D8000F0BD00BF9336EAA9EBE1F042F7B5384A5F
:101D9000106851686B4603C36A46364936480823C3
:101DA00004F054FB0446002833D10A25334A106856
:101DB00051686B4603C36A4631492F48082304F033
:101DC00045FB0446002849D00369B3F5702F45D878
:101DD000B0F8661040F2F63291423FD1294A0244EF
:101DE00002F15C018B4239D35C3B234900209E1AEF
:101DF000FFF784FF3246074604F164010020FFF735
:101E00007DFFA3689F4229D1E368984208BF00255F
:101E100024E00369B3F5702F27D8418B40F2F632E6
:101E2000914220D1174A024402F110018B4218D38B
:101E3000103B114900209D1AFFF760FF2A46064615
:101E400004F118010020FFF759FFA3689E4202D158
:101E5000E368984201D00D25A8E70025284603B085
:101E6000F0BD1025A2E70C25A0E70B259EE700BFDB
:101E7000AC650008DCFF0E0000000108B565000835
:101E800090FF0E000800FFF710B5037C044613B95D
:101E9000006804F0C3FA204610BD00000023BFF321
:101EA0005B8FC360BFF35B8FBFF35B8F8360BFF358
:101EB0005B8F7047BFF35B8F0068BFF35B8F70472A
:101EC00070B505460C30FFF7F5FF05F1080604462E
:101ED0003046FFF7EFFFA04206D930466D68FFF7A6
:101EE000E9FF2544281A70BD3046FFF7E3FF201AAA
:101EF000F9E7000070B50546406898B105F10800A3
:101F0000FFF7D8FF05F10C0604463046FFF7D2FF75
:101F10008442304694BF6D680025FFF7CBFF013C3B
:101F20002C44201A70BD000038B50C460546FFF75A
:101F3000C7FFA04210D305F10800FFF7BBFF044420
:101F40006868B4FBF0F100FB1144BFF35B8F012024
:101F5000AC60BFF35B8F38BD0020FCE72DE9F0419A
:101F6000144607460D46FFF7C5FF844228BF0446C6
:101F7000D4B1B84658F80C6B4046FFF79BFF30448D
:101F8000286040467E68FFF795FF331A9C4203D8CD
:101F90006C600120BDE8F0816B60A41B3B68AB6006
:101FA0002044E8600220F5E72046F3E738B50C4608
:101FB0000546FFF79FFFA04210D305F10C00FFF785
:101FC00079FF04446868B4FBF0F100FB1144BFF3EF
:101FD0005B8F0120EC60BFF35B8F38BD0020FCE716
:101FE0002DE9FF41884669460746FFF7B7FF6C4673
:101FF00006B204EBC6060025B44209D06268206828
:1020000008EB0501FFF7F6FB636808341D44F3E7AE
:1020100029463846FFF7CAFF284604B0BDE8F081DC
:10202000F8B505460C300F46FFF744FF05F10806EA
:1020300004463046FFF73EFFA042304688BF6C683A
:10204000FFF738FF201A386020B130462C68FFF7C0
:1020500031FF2044F8BD000073B5144606460D4616
:10206000FFF72EFF844228BF04460190DCB101A98E
:102070003046FFF7D5FF019B33B93268C5E902331B
:10208000C5E9002401200CE09C4238BF019428607F
:10209000019868608442F5D93368AB60241AEC601B
:1020A000022002B070BD2046FBE700002DE9FF4191
:1020B0000F466946FFF7D0FF6C4600B204EBC0053F
:1020C0000026AC4209D0D4F8048054F8081BB81993
:1020D0004246FFF78FFB4644F3E7304604B0BDE8C5
:1020E000F081000038B50546FFF7E0FF04460146E1
:1020F0002846FFF719FF204638BD000010B40268DB
:1021000054681A4623465DF8044B18470020704770
:102110000020704770470000002070470E20704775
:1021200000F5805090F8C800C0F3400070470000F0
:1021300000F5805090F9D0007047000000F5805005
:10214000C0F8CC1001207047F7B50C68BDF82070BE
:1021500014F0005470D10D7B082D6DD8302585F317
:1021600011884569AE6876010CD4AC68240108D4A6
:10217000AC6814F080545DD184F31188204603B01C
:10218000F0BD01240E6804F1180C002EB8BFF60053
:102190004FEA0C1CB4BF46F00406760545F80C6007
:1021A0000E680FFA84FC16F0804F18BF05EB0C1E6A
:1021B00005EB0C1C1EBFDEF8806146F00206CEF86F
:1021C00080610E7BCCF8846105EB04158E68C5F840
:1021D0008C614E68C5F88861DCF8805145F00105D6
:1021E000CCF8805100EB441641F268052E4405EB13
:1021F00044150544C6E9002308350E4601F10C0CD0
:1022000056F804EB45F804EB6645F9D1843436887A
:102210002E8000EB441407F00305267926F00B0608
:1022200035432571002484F31188009700F0FCFCED
:102230000120A4E70224A5E74FF0FF309FE700004C
:1022400013B500F580540191E06DFFF753FE1F2890
:102250000AD90199E06D2022FFF7C2FEA0F1200308
:102260005842584102B010BD0020FBE708B53023AA
:1022700083F3118800F58050C06DFFF70FFE002337
:1022800083F3118808BD0000002202608281426051
:102290008260704710B500220023C0E900230023AC
:1022A000044603810C30FFF7EFFF204610BD00000D
:1022B000F0B5054600F580500C4690F8C83013F094
:1022C000040FC3F3800108BF114661F3820304F1D8
:1022D000840680F8C83005EB461389B01B79D8070F
:1022E0002ED57AB319072DD46846FFF7D3FF05EB37
:1022F000441303F5835303F1180703AA1033186836
:102300005968144603C40833BB422246F7D1186803
:1023100020609B88A380DDE90E23CDE90023012303
:10232000ADF808302B686946DB6B2846984705EB0B
:1023300046152B791A075CBF43F008032B7101E0A7
:10234000002AF4D109B0F0BD2DE9F0479A4688B0D3
:10235000074688469146302383F3118807F5805459
:102360006846FFF797FFE06DFFF7AAFD1F282AD9FF
:10237000E06D20226946FFF7B5FE202823D103AD8A
:10238000444605AB2E4603CE9E4220606160354632
:1023900004F10804F6D130682060B388A380DDE939
:1023A0000023C9E90023BDF80830AAF80030002353
:1023B00083F3118853464A464146384608B0BDE883
:1023C000F04700F01FBC002080F3118808B0BDE882
:1023D000F08700002DE9F84F0023C0E90133254BB9
:1023E000044640F8183B0F46FFF74EFF04F1280063
:1023F000FFF750FF04F1480804F5825546460835BA
:1024000030462036FFF746FFAE42F9D104F580553D
:102410004FF480534FF00009C5E91339C5F84880DF
:102420000123EE6504F5875804F58456C5F85490E9
:1024300085F8583085F86030083608F108084FF004
:10244000000A4FF0000B46E908ABA6F11800FFF7B1
:102450001BFF203646F8289C4645F4D185F8D070FD
:1024600017B1054800F0B8FB044B63612046BDE896
:10247000F88F00BFE8650008C065000800640040F0
:1024800010B5044B197804464A1C1A70FFF7A2FFD6
:10249000204610BD644B00202DE9F047002950D0A4
:1024A000294B2A4FB7FBF1F599428CBF0A23112320
:1024B000581EB5FBF3FC03FB1C53C4B22BB102281E
:1024C0000346F5D80020BDE8F0870CF1FF36B6F5DD
:1024D000806FF7D2C4EBC40E0EF103034FEAE30999
:1024E000C3F3C703A4EB030809F1010A4FF47A759B
:1024F0005FFA88F009FB05555AFA88F8B5FBF8F53C
:10250000B5F5617FC1BF0EF1FF33C3F3C703E01A16
:10251000C0B25C1C50FA84F40CFB04F4B7FBF4F476
:10252000A142CFD1013BDBB20F2BCBD80138C0B2D7
:102530000728C7D80021107116809170D370012030
:10254000C1E70846BFE700BF3F420F0080DE8002C0
:1025500070B505460E464FF47A746B695B6803F0FC
:102560000103B34207D04FF47A7002F0C5F8013C82
:10257000F3D1204670BD0120FCE7000030B5426970
:10258000936913F0700F16D000230B4C936103F185
:10259000840200EB421211794D0709D5890707D54E
:1025A000416954F823508D60117941F00401117193
:1025B0000133032BEBD130BDD465000873B51D4644
:1025C000436916469A68D207044609D59A680121DC
:1025D0009960C2F34002CDE900650021FFF768FE73
:1025E00063699A68D1050BD59A684FF48071996038
:1025F000C2F34022CDE9006501212046FFF758FED5
:1026000063699A68D2030BD59A684FF48031996058
:10261000C2F34042CDE9006502212046FFF748FEA3
:1026200004F58053D3F8CC0010B103681B699847B8
:10263000204602B0BDE87040FFF7A0BFF8B50446E1
:102640004669002972D106F10C073868800770D0FE
:1026500006EB01153868D5F8B00110F0040FD5F875
:10266000B0011ABFC00840F00040400DA061D5F88D
:10267000B0C11CF0020F1CBF40F08040A061D5F833
:10268000B40106EB011100F00F0084F82400D1F82A
:10269000B8012077D1F8B801000A6077D1F8B80105
:1026A000000CA077D1F8B801000EE077D1F8BC019A
:1026B00084F82000D1F8BC01000A84F82100D1F888
:1026C000BC01000C84F82200D1F8BC11090E84F87A
:1026D00023103821396004F1340004F1180104F1A9
:1026E000240551F8046B40F8046BA942F9D109881C
:1026F0000180C4E90A2321460023238651F8283BA0
:102700002046DB6B984704F5805393F8C820D3F834
:10271000CC0042F0040283F8C82010B103681B69A2
:1027200098472046BDE8F840FFF728BF06F110079C
:102730008BE7F8BD10B5044600F056FA02460B468A
:1027400052EA030102D0013A63F100030449086828
:1027500020B12146BDE81040FFF770BF10BD00BF9B
:10276000604B0020F0B5302181F31188DFF848C0BC
:1027700000F583510831002404F1840500EB451570
:102780002E7977070ED4F6060CD5D1E9007697425C
:102790009E4107D246695CF82470B7602E7946F0F6
:1027A00004062E710134032C01F12001E4D1002331
:1027B00083F31188F0BD00BFD465000808B530234D
:1027C00083F31188FFF7DAFE002383F3118808BD35
:1027D000F8B543690546986800F0E050B0F1E05F55
:1027E0000F4621D0F8B1302383F3118805F58354C7
:1027F0001034002606F1840305EB43131B791A07F6
:1028000006D50136032E04F12004F3D1012007E0A0
:102810005B07F6D42146384600F040FA0028F0D194
:10282000002383F31188F8BD0120FCE708B53023AD
:1028300083F3118800F58050C06DFFF741FB002342
:1028400083F3118843090CBF0120002008BD00005C
:10285000F8B51D46002313700F4606461446FFF7D1
:10286000E5FF80F00100387025B129463046FFF7BA
:10287000AFFF2070F8BD00002DE9B8410C461546A9
:102880001F46804600F0B0F90B462178024609B990
:10289000287850B14046FFF765FFFFF78FFF3B46B2
:1028A0002A462146FFF7D4FF0120BDE8B881000089
:1028B00070B5302686F31188174B1A6C42F00072FF
:1028C0001A641A6A42F000721A621A6A22F00072DE
:1028D0001A62002383F3118800F5805494F8C830FD
:1028E00013F0010516D1A9B186F311880321132035
:1028F00001F0C8F90321142001F0C4F903211520C7
:1029000001F0C0F994F8C83043F0010384F8C830EE
:1029100085F3118870BD00BF003802402DE9F047F3
:1029200000F5805588B095F8D030012B04468846D4
:10293000164600F28180814F57F823200AB947F8E4
:102940002300D7F800A0C4F80C802674BAF1000F59
:1029500064D095F8D030012B70D001212046FFF7CC
:10296000A7FF302383F311886269136823F0020301
:1029700013606269136843F0010313606369002701
:102980005F6187F3118801212046FFF7E1FD0028F0
:1029900000F09580E86DFFF781FA04F58359BA4697
:1029A00009F10809202200216846FEF749FF02A824
:1029B000FFF76AFCCDF818A06A4609EB07030DF192
:1029C000180E9446BCE80300F4451860596062464E
:1029D00003F10803F5D1DCF80000186020379CF8FB
:1029E00004201A71602FDDD195F8C8306FF382038F
:1029F000002785F8C8306A4641462046ADF8007089
:102A0000ADF802708DF80470FFF746FD636948BBAE
:102A10004FF400421A6008B0BDE8F08741F2D800D8
:102A200003F0BCFC814610B15146FFF7D3FCC7F858
:102A30000090B9F1000F8CD10020ECE738680368F2
:102A40001B6B98470146002887D13868FFF730FF95
:102A50003868036832465B684146984700287FF42F
:102A60007CAFE9E761221A609DF802309DF80320EF
:102A70001B06120402F4702203F040731343BDF8E6
:102A80000020C2F3090213439DF804201205022E10
:102A900002F4E0020CBF4FF00041002113436269D1
:102AA0000B43D361636913225A616269136823F08F
:102AB0000103136039462046FFF74AFD08B96369F0
:102AC000A6E795F8D03093BB6169D1F8002242F0B7
:102AD0000102C1F800226169D1F8002222F47C527F
:102AE00022F00E02C1F800226169D1F8002242F4FE
:102AF0006062C1F800226269C2F814326269C2F8E9
:102B00000432626941F6FF71C2F80C126269C2F8C0
:102B100040326269C2F8443263690122C3F81C2260
:102B20006269D2F8003223F00103C2F8003295F84E
:102B3000C83043F0020385F8C8306CE7604B0020D2
:102B400008B500F051F850EA0103024602D0421ED7
:102B500061F10001044B186810B10B46FFF72EFD20
:102B6000BDE8084001F064B8604B002008B50020C3
:102B7000FFF7E0FDBDE8084001F05AB808B50120B4
:102B8000FFF7D8FDBDE8084001F052B800B59BB092
:102B9000EFF3098168226846FEF72CFEEFF3058308
:102BA000014B9B6BFEE700BF00ED00E008B5FFF7AF
:102BB000EDFF000000B59BB0EFF309816822684685
:102BC000FEF718FEEFF30583014B5B6BFEE700BFDA
:102BD00000ED00E0FEE700000FB408B5029801F038
:102BE00031FDFEE702F0B4B902F096B913B56C46B8
:102BF00084E80600031D94E8030083E80500012033
:102C000002B010BD73B58568019155B11B885B0793
:102C100007D4D0E900369B6B9847019AC1B2304681
:102C2000A847012002B070BDF0B5866889B005469E
:102C30000C465EB1BDF838305B070AD4D0E90037E6
:102C40009B6B98472246C1B23846B047012009B075
:102C5000F0BD00220023CDE900230023ADF80830A9
:102C60000A4603AB01F10806106851681C4603C40C
:102C70000832B2422346F7D1106820609288A280C1
:102C8000FFF7B2FF0423ADF808302B68CDE900014F
:102C9000DB6B694628469847D8E7000030B50368E3
:102CA0000968DD0FB5EBD17F23F0604421F060426D
:102CB0004FEAD1700BD0002BB8BFA40C0029B8BFCD
:102CC000920C944202D034BF0120002030BD9442C7
:102CD00005D1C1F38070C3F380738342F6D194426F
:102CE0002CBF00200120F1E72DE9F041456A15B91C
:102CF0004162BDE8F0814B6823F06047C3F38A4628
:102D00004FEAD37EC3F3807816EA230638BF3E46E7
:102D1000AC462B465A68BEEBD27F22F060440AD004
:102D2000002A18DAA40CB44217D19D420FD10D60CD
:102D3000DEE71346EEE7A74207D102F08044C2F374
:102D4000807242450BD054B1EFE708D2EDE7CCF8E2
:102D500000100B60CDE7B44201D0B442E5D81A6848
:102D60009C46002AE5D11960C3E700002DE9F04731
:102D7000089D01F007044FEAD508224405F0070535
:102D800000EBD1004FF47F49944201D1BDE8F087B8
:102D900004F0070705F0070A57453E4638BF564678
:102DA000C6F10806111B8E4228BF0E46E10808EB4B
:102DB000D50E415C13F80EC0B94029FA06F721FA86
:102DC0000AF1FFB28CEA010147FA0AF739408CEAAE
:102DD000010C03F80EC034443544D5E780EA0120E5
:102DE000082341F2210201B24000002980B203F120
:102DF000FF33B8BF504013F0FF03F4D17047000019
:102E000038B50C468D18A54200D138BD14F8011B09
:102E1000FFF7E4FFF7E7000042684AB11368436038
:102E20004389818901339BB29942438138BF8381B1
:102E30001046704770B588B0202204460D4668469B
:102E40000021FEF7FDFC20460495FFF7E5FF024652
:102E500058B16B46054608AE1C4603CCB442286008
:102E60006960234605F10805F6D1104608B070BD2B
:102E7000082817D909280CD00A280CD00B280CD008
:102E80000C280CD00D280CD00E2814BF4020302068
:102E900070470C207047102070471420704718208E
:102EA0007047202070470000082817D90C280CD93B
:102EB00010280CD914280CD918280CD920280CD982
:102EC00030288CBF0F200E207047092070470A2041
:102ED00070470B2070470C2070470D207047000092
:102EE0002DE9F843078C072F04461ED9D0E9029834
:102EF00000254FF6FF73C5F12006A5F1200029FA41
:102F000005F108FA06F628FA00F031430143C9B288
:102F10001846FFF763FF0835402D0346EBD1E16902
:102F20003A46BDE8F843FFF76BBF4FF6FF70BDE8C8
:102F3000F883000010B54B6823B9CA8A63F309020D
:102F4000CA8210BD04691A681C600361C38A013B10
:102F5000C3824A60EFE700002DE9F84F1D46CB8A97
:102F60000F46C3F309010529814692460B4630D02E
:102F70000020AAB207F11A049EB2042E1FFA80F8AC
:102F80000FD8904503F1010306D3FB8A0A4462F38C
:102F90000903FB8201201AE01AF80060E6540130B0
:102FA000EAE79045F1D2A1F1050B1C237C68BBFB3D
:102FB000F3F203FB12BB1FFA8BF6002C45D14846F7
:102FC000FFF72AFF044638B978606FF00200BDE8C9
:102FD000F88F4FF00008E6E7002606607860ADB293
:102FE0004FF0000B454510D90AEB0803221D13F8DA
:102FF000011B9155B1B208F101081B291FFA88F88D
:103000002BD0454506F10106F1D8FB8AC3F309022E
:10301000154465F30903BCE7013292B21C462368EC
:10302000002BF9D16B1F0B441C21B3FBF1F30133CF
:103030009BB29A42D3D2BBF1000FD0D14846FFF7E2
:10304000EBFE20B9C4F800B0BFE70122E7E7C0F803
:1030500000B05E4620600446C1E74545D5D94846E4
:10306000FFF7DAFE08B92060AFE7C0F800B000262D
:1030700020600446B6E700002DE9F04F2DED028BED
:103080001C4683B05B69019207468846002B00F01E
:103090009A80238C2BB1E269002A00F09480072BE0
:1030A00035D807F10C00FFF7B7FE054638B96FF0C9
:1030B0000205284603B0BDEC028BBDE8F08F142258
:1030C0000021FEF7BDFB228CE16905F10800FEF747
:1030D00091FB208C013080B2FFF7E6FEFFF7C8FEBF
:1030E000013880B22084013028746369228C1B78F7
:1030F0002A4403F01F0363F03F0348F000411372BA
:10310000384669602946FFF7EFFD0125D1E700F158
:103110000C034FF0000908EE103A4FF0800A4E46BB
:103120004D4618EE100AFFF777FE83460028BED002
:1031300014220021FEF784FB002E3AD1019BABF84C
:10314000083002220BF1080E1FFA82FC0CF101007C
:10315000BCF1060F218C80B201D88E422BD3FFF731
:10316000A3FEFFF785FE62691278013802F01F02A4
:103170008E4208BF4FF0400A42EA49121BFA80F122
:103180004AEA020A013048F0004281F808A08BF8B0
:103190001000CBF8042059463846FFF7A5FD238CD4
:1031A0000135B3422DB289F001094FF0000AB8D1C0
:1031B0007FE70022C6E7E169895D0EF8021001365B
:1031C000B6B20132C0E76FF0010572E7F8B51546F7
:1031D0000E463022002104461F46FEF731FB069BB7
:1031E0006360B5F5001F079BA76034BF6A094FF6FF
:1031F000FF72A36297B2E66104F1100000239A42C5
:1032000006D800230360A782E3822383E360F8BD2E
:103210000660013330462036F1E7000003781BB921
:103220004BB2002BC8BF0170704700000078704798
:10323000F8B50C46C969074611B9238C002B37D164
:10324000257E1F2D34D8387828BB228C072A2CD80D
:10325000268A36F003032BD14FF6FF70FFF7D0FD1F
:1032600020F001003102400441EA0561400C41EACE
:1032700040254FF6FF72234629463846FFF7FCFEED
:10328000002807DD626913780133DBB21F2B88BF8A
:1032900000231370F8BD218A2D0645EA0125054358
:1032A0002046FFF71DFE0246E5E76FF00300F1E759
:1032B0006FF00100EEE7000070B58AB004461646D4
:1032C0000021282268461D46FEF7BAFABDF83830BC
:1032D000ADF810300F9B05939DF840308DF81830F5
:1032E000119B07936946BDF84830ADF82030204661
:1032F000CDE90265FFF79CFF0AB070BD2DE9F041F2
:10330000D36905460C4616460BB9138C5BBB377E5A
:103310001F2F28D895F80080B8F1000F26D030462E
:10332000FFF7DEFD3378210241EAC33141EA0801AB
:10333000338A41EA076141EA03410246334641F0DC
:1033400080012846FFF798FE00280ADD3378012B1C
:1033500007D1726913780133DBB21F2B88BF0023BA
:103360001370BDE8F0816FF00100FAE76FF0030021
:10337000F7E70000F0B58BB004460D461746002174
:10338000282268461E46FEF75BFA9DF84C305A1E0E
:10339000534253418DF800309DF84030ADF8103065
:1033A000119B05939DF848308DF81830149B0793B6
:1033B0006A46BDF85430ADF8203029462046CDE9A4
:1033C0000276FFF79BFF0BB0F0BD0000406A00B132
:1033D00004307047436A1A68426202691A600361E6
:1033E000C38A013BC38270472DE9F041D0F82080A9
:1033F000194E14461D464146002709B9BDE8F08123
:10340000D1E90223A21A65EB0303964277EB03038B
:103410001ED2036A8B420DD1FFF78CFD036A1B6835
:10342000036203690B60C38A0161016A013BC382C5
:103430008846E2E7FFF77EFD0B68C8F800300369B5
:103440000B60C38A0161013BC382D8F80010D4E746
:1034500088460968D1E700BF80841E002DE9F04F3F
:103460008BB00D46DDF8509014469B4680460028F0
:1034700000F01981B9F1000F00F01581531E3F2BA8
:1034800000F21181012A03D1BBF1000F40F00B8142
:103490000023CDE90833B8F81430B5EBC30F4FEA79
:1034A000C30703D300200BB0BDE8F08F2B199F4258
:1034B000D8F80C303ABF7F1BFFB227461BB9D8F8AB
:1034C0001030002B7AD0272D4ED8C5F12806B742F0
:1034D0004FF000032CBFF6B23E4600932946D8F8C1
:1034E000080008AB3246FFF741FCA7EB060A35445B
:1034F0005FFA8AFAB8F8143003F10053053BDB0099
:103500000493D8F80C3003932821039B13B1BAF12C
:10351000000F2CD1D8F8100040B1BAF1000F05D03F
:10352000009608AB5246691AFFF720FC38B2002F0C
:10353000B8D066070AD00AAB03EBD401624211F897
:10354000083C02F00702134101F8083C082C3CD962
:10355000102C40F2B580202C40F2B780BBF1000F58
:1035600000F09C80082334E0BA460026C2E7049BA2
:10357000E02B28BFE02306930B44AB42059314D9FC
:103580005A1B03980096924534BF5246D2B2691A2C
:1035900008AB04300792FFF7E9FB079A1644AAEB41
:1035A000020A1544F6B25FFA8AFA049B069A059954
:1035B0009B1A0493039B1B680393A6E70093D8F818
:1035C000080008AB3A462946AEE7BBF1000F13D01E
:1035D0000123B4EBC30F6CD0082C12D89DF8203017
:1035E000621E23FA02F2D50706D54FF0FF3202FA27
:1035F00004F423438DF820309DF8203089F8003002
:1036000051E7102C12D8BDF82030621E23FA02F2C6
:10361000D10706D54FF0FF3202FA04F42343ADF888
:103620002030BDF82030A9F800303CE7202C0FD81E
:103630000899631E21FA03F3DA0705D54FF0FF322C
:1036400002FA04F40C430894089BC9F800302AE7F6
:10365000402C2BD0DDE90865611EC4F12102A4F1E4
:10366000210326FA01F105FA02F225FA03F31143C8
:103670001943CB0712D50122A4F12003C4F1200184
:1036800002FA03F322FA01F1A240524243EA010393
:1036900063EB430332432B43CDE90823DDE90823E1
:1036A000C9E90023FFE66FF00100FCE66FF00800B7
:1036B000F9E6082CA0D9102CB3D9202CEED8C3E7FA
:1036C000BBF1000FADD0022383E7BBF1000FBBD0ED
:1036D00004237EE730B5012A144638BF0124402C6C
:1036E00085B028BF40240025012ACDE9025518D80D
:1036F0001B788DF8083063070AD004AB03EBD405C0
:10370000624215F8083C02F00702934005F8083CB5
:10371000009103462246002102A8FFF727FB05B0CF
:1037200030BD082AE4D9102A03D81B88ADF8083028
:10373000E1E7202A8DBFD3E900231B680293CDE97E
:103740000223D8E710B5CB681BB98B600B618B8265
:1037500010BD04691A681C600361C38A013BC382FF
:10376000CA60F0E703064CBFC0F3C03002207047C8
:1037700008B50246FFF7F6FF022806D15306C2F34A
:103780000F2001D100F0030008BDC2F30740FBE7A2
:103790002DE9F04F93B0CDE903230A6804461046A3
:1037A000FFF7E0FF022814BFC2F306260026002A16
:1037B0000D46824680F2F28112F0C04940F0EE815F
:1037C000097B002900F0EA81022803D02378B34264
:1037D00040F0E781C2F304630693104602F07F03D2
:1037E0000593FFF7C5FF059B29444FEA834848EA44
:1037F0000A4848EA4668CE7800230022CDE908232B
:10380000F309834648EA0008029367D0059B0093BA
:1038100002466768534608A92046B847002800F0CA
:10382000C381276A4FB9414604F10C00FFF702FB40
:10383000074690B96FF0020054E03B6998450DD0FF
:103840003F68002FF9D1414604F10C00FFF7F2FA6E
:1038500007460028EED0236A3B60276297F817C01E
:1038600006F01F08CCF3840CACEB08001FFA80FEB6
:103870000028B8BF0EF12000A8EB0C031FFA83FE4E
:10388000D7E90221B8BF00B2002B0793BEBF0EF1EB
:1038900020031BB2079352EA010338D0039BDFF8E1
:1038A00024E39A1A049B4FF0000C63EB0101964548
:1038B0007CEB01032BD36B7B97F81AE0734519D18E
:1038C000029B002B78D0012821DC7868F8B9DFF85A
:1038D000F0C2944570EB010316D337E0276A27B98D
:1038E0006FF00C0013B0BDE8F08F3B699845B5D080
:1038F0003F68F4E7B24890427CEB010301D300201B
:10390000F0E7029B002BFAD0079B0F2B17DCFA7D08
:10391000B30002F0030203F07C031343FB75394646
:103920002046FFF707FB6B7BBB76029B3BB9FB7D19
:10393000C3F38402013262F38603FB75D0E76A7B2E
:10394000BB7E9A42DBD1029B002B35D0B309022B00
:1039500032D0039BBB60049BFB60142200210DA8A6
:10396000FDF76EFF039B0A93049B0B932B1D0C9397
:103970002B7BADF83EB0013BDBB2ADF83C30069B93
:103980008DF84230059B8DF8433094F82C308DF83B
:1039900040A083F001038DF844308DF84180A36886
:1039A0000AA920469847FB7DC3F38403013303F043
:1039B0001F039B02FB82A2E7FB7DC6F34012B2EB22
:1039C000D31F40F0F480C3F38403434540F0F280FA
:1039D000029A2B7BB609002A4DD0F2075DD4032B47
:1039E00040F2EB80039BBB60049BFB602B7BAE1D16
:1039F000033BDBB23246394604F10C00FFF7ACFA68
:103A000000280CDA39462046FFF794FAFB7DC3F311
:103A10008403013303F01F039B02FB820AE7DDE905
:103A20000884AB883B834FF6FF73C9F12000A9F1EE
:103A3000200228FA09F104FA00F0014324FA02F204
:103A400011431846C9B2FFF7C9F909F10809B9F1DC
:103A5000400F0346E9D1B8822A7B033AD2B23146FD
:103A6000FFF7CEF9FB7DB882DA43C2F3C01262F3EE
:103A7000C713FB7543E786B92E1D013BDBB2324607
:103A8000394604F10C00FFF767FA0028BADB2A7BFD
:103A9000B88A013AD2B23146E2E7F98AC1F30901A4
:103AA000013B0429DAB25BD8281D002307F11B066D
:103AB0009A4208D910F801CB06F801C00131013350
:103AC0000529DBB2F4D103990A9104990B91934231
:103AD00007F11B010C9138BF043379680D9134BF95
:103AE00055FA83F300230E93FB8AADF83EB0C3F37F
:103AF00009031A44069B8DF84230059B8DF843302C
:103B000094F82C30ADF83C2083F001038DF844305C
:103B100000238DF840A08DF841807B602A7BB88A15
:103B2000013A291DFFF76CF93B8BB882834203D120
:103B3000A3680AA92046984720460AA9FFF702FE73
:103B4000FB7DBA8AC3F38403013303F01F039B0296
:103B5000FB823B8B9A420CBF00206FF01000C1E645
:103B60007B68002BAFD0052001E01C3033461E6877
:103B7000002EFAD1091A081D2E1D184401EB090C5C
:103B8000BCF11B0F5FFA89F39DD89A429BD916F8B6
:103B9000013B00F8013B09F10109EFE76FF0090073
:103BA000A0E66FF00A009DE66FF00B009AE66FF05A
:103BB0000D0097E66FF00E0094E66FF00F0091E6AF
:103BC00040420F0080841E00EFF3098305494A6BD1
:103BD00022F001024A63683383F30988002383F3E8
:103BE0001188704700EF00E0302080F3118862B642
:103BF0000C4B0D4AD96821F4E0610904090C0A4311
:103C0000DA60D3F8FC20094942F08072C3F8FC2046
:103C10000A6842F001020A602022DA7783F8220063
:103C2000704700BF00ED00E00003FA05001000E05F
:103C300010B5302383F311880E4B5B6813F40063D7
:103C400014D0F1EE103AEFF30984683C4FF0807322
:103C5000E361094BDB6B236684F3098800F0BCFC4D
:103C600010B1064BA36110BD054BFBE783F3118830
:103C7000F9E700BF00ED00E000EF00E03F030008BF
:103C80004203000800F1604303F561430901C9B232
:103C900083F80013012200F01F039A4043099B00A0
:103CA00003F1604303F56143C3F880211A60704754
:103CB000026843681143016003B118477047000070
:103CC00013B5446BD4F894341A681178042915D1CB
:103CD000217C022912D11979128901238B401342C8
:103CE0000CD101A904F14C0001F09CFFD4F89444DC
:103CF000019B21790246206800F0D0F902B010BD86
:103D0000143001F01FBF00004FF0FF33143001F0FA
:103D100019BF00004C3001F0F1BF00004FF0FF333D
:103D20004C3001F0EBBF0000143001F0EDBE00009C
:103D30004FF0FF31143001F0E7BE00004C3001F0CD
:103D4000BDBF00004FF0FF324C3001F0B7BF0000A4
:103D50000020704710B5D0F894341A6811780429FF
:103D6000044617D1017C022914D1597952890123C3
:103D70008B4013420ED1143001F080FE024648B150
:103D8000D4F894444FF4807361792068BDE8104002
:103D900000F072B910BD0000406BFFF7DBBF000000
:103DA000704700007FB5124B036000234360C0E9F9
:103DB0000233012502260F4B05740446029001933D
:103DC00000F18402294600964FF48073143001F00C
:103DD00031FE094B0294CDE9006304F523724FF4E0
:103DE0008073294604F14C0001F0F8FE04B070BD68
:103DF00028660008993D0008C13C00080B68302285
:103E000082F311880A7903EB820290614A790932C0
:103E100043F822008A7912B103EB820398610223EE
:103E2000C0F894140374002080F3118870470000D8
:103E300038B5037F044613B190F85430ABB9201D58
:103E400001250221FFF734FF04F1140025776FF0FC
:103E5000010100F079FC84F8545004F14C006FF03B
:103E60000101BDE8384000F06FBC38BD10B501213C
:103E700004460430FFF71CFF0023237784F85430F6
:103E800010BD000038B504460025143001F0EAFDED
:103E900004F14C00257701F0B9FE201D84F8545040
:103EA0000121FFF705FF2046BDE83840FFF752BF6C
:103EB00090F8443003F06003202B07D190F84520A0
:103EC000212A4FF0000303D81F2A06D8002070478C
:103ED000222AFBD1C0E90E3303E0034A82630722A2
:103EE000C2630364012070471D23002037B5D0F85A
:103EF00094341A681178042904461AD1017C0229E5
:103F000017D11979128901238B40134211D100F185
:103F10004C05284601F03AFF58B101A9284601F0A6
:103F200081FED4F89444019B21790246206800F078
:103F3000B5F803B030BD0000F0B500EB810385B0EB
:103F40009E6904460D46FEB1302383F3118804EBCD
:103F50008507301D0821FFF7ABFEFB685B691B6816
:103F600006F14C001BB1019001F06AFE019803A913
:103F700001F058FE024648B1039B2946204600F056
:103F80008DF8002383F3118805B0F0BDFB685A69F2
:103F90001268002AF5D01B8A013B1340F1D104F1CD
:103FA0004402EAE7093138B550F82140DCB130234A
:103FB00083F31188D4F894241368527903EB8203B5
:103FC000DB689B695D6845B104216018FFF770FEEE
:103FD000294604F1140001F05BFD2046FFF7BAFE0C
:103FE000002383F3118838BD7047000001F0D0B87A
:103FF000012303700023C0E90133C36183620362BC
:10400000C36243620363704738B50446302383F3C9
:1040100011880025C0E90355C0E90555416001F04C
:10402000C7F80223237085F31188284638BD0000A5
:1040300070B500EB810305465069DA600E46144600
:1040400018B110220021FDF7FBFBA06918B1102266
:104050000021FDF7F5FB31462846BDE8704001F030
:1040600071B90000826802F0011282600022C0E98A
:104070000422826101F0F2B9F0B400EB81044789B7
:10408000E4680125A4698D403D43458123600023F8
:10409000A2606360F0BC01F00DBA0000F0B400EB68
:1040A00081040789E468012564698D403D430581E9
:1040B00023600023A2606360F0BC01F087BA0000B7
:1040C00070B50223002504460370C0E90255C0E91B
:1040D0000455C564856180F8345001F0CFF86368F9
:1040E0001B6823B129462046BDE87040184770BDC3
:1040F0000378052B10B504460AD080F8503005230C
:10410000037043681B680BB1042198470023A36028
:1041100010BD00000178052906D190F850204368B1
:1041200002701B6803B118477047000070B590F823
:104130003430044613B1002380F8343004F14402D3
:10414000204601F0ADF963689B68B3B994F8443038
:1041500013F0600535D00021204601F04DFC002110
:10416000204601F03FFC63681B6813B1062120461E
:104170009847062384F8343070BD204698470028BD
:10418000E4D0B4F84A30E26B9A4288BFE36394F912
:104190004430E56B002B4FF0300380F20381002D9B
:1041A00000F0F280092284F8342083F31188002182
:1041B000D4E90E232046FFF771FF002383F3118813
:1041C000DAE794F8452003F07F0343EA022340F244
:1041D0000232934200F0C58021D8B3F5807F48D0E9
:1041E0000DD8012B3FD0022B00F09380002BB2D1D1
:1041F00004F14C02A2630222E2632364C1E7B3F537
:10420000817F00F09B80B3F5407FA4D194F84630C5
:10421000012BA0D1B4F84C3043F0020332E0B3F5E7
:10422000006F4DD017D8B3F5A06F31D0A3F5C063A0
:10423000012B90D8636894F846205E6894F8471084
:10424000B4F848302046B047002884D04368A363C0
:104250000368E3631AE0B3F5106F36D040F602420C
:1042600093427FF478AF5C4BA3630223E3630023A4
:10427000C3E794F84630012B7FF46DAFB4F84C30AF
:1042800023F00203C4E90E55A4F84C30256478E706
:10429000B4F84430B3F5A06F0ED194F8463084F8EA
:1042A0004E30204601F042F863681B6813B10121CB
:1042B00020469847032323700023C4E90E339CE76C
:1042C00004F14F03A3630123C3E72378042B10D128
:1042D000302383F311882046FFF7C4FE85F311884D
:1042E0000321636884F84F5021701B680BB120468E
:1042F000984794F84630002BDED084F84F300423E2
:10430000237063681B68002BD6D002212046984793
:10431000D2E794F848301D0603F00F0120460AD575
:1043200001F0B0F8012804D002287FF414AF2B4B21
:104330009AE72B4B98E701F097F8F3E794F84630AB
:10434000002B7FF408AF94F8483013F00F01B3D07E
:104350001A06204602D501F063FBADE701F056FBDB
:10436000AAE794F84630002B7FF4F5AE94F8483075
:1043700013F00F01A0D01B06204602D501F03CFB34
:104380009AE701F02FFB97E7142284F8342083F397
:1043900011882B462A4629462046FFF76DFE85F3F5
:1043A0001188E9E65DB1152284F8342083F3118881
:1043B0000021D4E90E232046FFF75EFEFDE60B2226
:1043C00084F8342083F311882B462A462946204658
:1043D000FFF764FEE3E700BF586600085066000878
:1043E0005466000838B590F834300446002B3ED0AF
:1043F000063BDAB20F2A34D80F2B32D8DFE803F0AD
:1044000037313108223231313131313131313737C1
:10441000C56BB0F84A309D4214D2C3681B8AB5FB05
:10442000F3F203FB12556DB9302383F311882B4649
:104430002A462946FFF732FE85F311880A2384F8BD
:1044400034300EE0142384F83430302383F31188A1
:1044500000231A4619462046FFF70EFE002383F379
:10446000118838BD036C03B198470023E7E70021AA
:10447000204601F0C1FA0021204601F0B3FA63683A
:104480001B6813B10621204698470623D7E7000092
:1044900010B590F83430142B044629D017D8062BC9
:1044A00005D001D81BB110BD093B022BFBD8002160
:1044B000204601F0A1FA0021204601F093FA63683A
:1044C0001B6813B1062120469847062319E0152BD7
:1044D000E9D10B2380F83430302383F31188002393
:1044E0001A461946FFF7DAFD002383F31188DAE74D
:1044F000C3689B695B68002BD5D1036C03B19847F7
:10450000002384F83430CEE7002303758268036902
:104510001B6899689142FBD25A6803604260106040
:104520005860704700230375826803691B689968A7
:104530009142FBD85A68036042601060586070472F
:1045400008B50846302383F311880B7D032B05D073
:10455000042B0DD02BB983F3118808BD8B69002281
:104560001A604FF0FF338361FFF7CEFF0023F2E7BD
:10457000D1E9003213605A60F3E70000FFF7C4BFCF
:10458000054BD9680875186802681A6053600122E3
:104590000275D860FBF7BEBE704B002030B50C4BE7
:1045A000DD684B1C87B004460FD02B46094A68468D
:1045B00000F05EF92046FFF7E3FF009B13B1684669
:1045C00000F060F9A86907B030BDFFF7D9FFF9E73F
:1045D000704B002041450008044B1A68DB68906866
:1045E0009B68984294BF002001207047704B0020C8
:1045F000084B10B51C68D86822681A605360012205
:104600002275DC60FFF78EFF01462046BDE81040B2
:10461000FBF780BE704B002038B5074C07490848AF
:10462000012300252370656001F0E8FB022323705D
:1046300085F3118838BD00BFD84D002060660008A2
:10464000704B002008B572B6044B186500F046FCAC
:1046500000F0FCFC024B03221A70FEE7704B0020B6
:10466000D84D002000F044B9034A516853685B1AE2
:104670009842FBD8704700BF001000E08B60022317
:1046800008618B82084670478368A3F1840243F86F
:10469000142C026943F8442C426943F8402C094A1F
:1046A00043F8242CC26843F8182C022203F80C2C7F
:1046B000002203F80B2C044A43F8102CA3F120002D
:1046C000704700BF2D030008704B002008B5FFF7AE
:1046D000DBFFBDE80840FFF751BF0000024BDB687D
:1046E00098610F20FFF74CBF704B0020302383F3FD
:1046F0001188FFF7F3BF000008B50146302383F3AC
:1047000011880820FFF74AFF002383F3118808BDB2
:10471000064BDB6839B1426818605A601360436029
:104720000420FFF73BBF4FF0FF307047704B002075
:104730000368984206D01A68026050609961184672
:10474000FFF71CBF7047000038B504460D462068CF
:10475000844200D138BD036823605C608561FFF747
:104760000DFFF4E710B503689C68A2420CD85C68A2
:104770008A600B604C602160596099688A1A9A605F
:104780004FF0FF33836010BD1B68121BECE7000085
:104790000A2938BF0A2170B504460D460A26601959
:1047A00001F026FB01F012FB041BA54203D8751C87
:1047B0002E460446F3E70A2E04D9BDE870400120D6
:1047C00001F05CBB70BD0000F8B5144B0D46D9611B
:1047D00003F1100141600A2A1969826038BF0A2278
:1047E000016048601861A818144601F0F3FA0A271E
:1047F00001F0ECFA431BA342064606D37C1C2819A1
:1048000001F0F6FA27463546F2E70A2F04D9BDE84B
:10481000F840012001F032BBF8BD00BF704B002012
:10482000F8B506460D4601F0D1FA0F4A134653F883
:10483000107F9F4206D12A4601463046BDE8F84027
:10484000FFF7C2BFD169BB68441A2C1928BF2C4698
:10485000A34202D92946FFF79BFF2246314603486F
:10486000BDE8F840FFF77EBF704B0020804B002072
:1048700010B4C0E9032300235DF8044B4361FFF744
:10488000CFBF000010B5194C236998420DD0D0E974
:104890000032816813605A609A680A449A60002363
:1048A00003604FF0FF33A36110BD2346026843F855
:1048B000102F53600022026022699A4203D1BDE8A2
:1048C000104001F08FBA936881680B44936001F047
:1048D0007DFA2269E1699268441AA242E4D911443E
:1048E000BDE81040091AFFF753BF00BF704B00200E
:1048F0002DE9F047DFF8BC8008F110072C4ED8F8FE
:10490000105001F063FAD8F81C40AA68031B9A42C1
:104910003ED81444D5E900324FF00009C8F81C40D5
:1049200013605A60C5F80090D8F81030B34201D136
:1049300001F058FA89F31188D5E9033128469847E0
:10494000302383F311886B69002BD8D001F03EFA35
:104950006A69A0EB04094A4582460DD2022001F0A3
:104960008DFA0022D8F81030B34208D151462846BB
:10497000BDE8F047FFF728BF121A2244F2E712EB16
:10498000090938BF4A4629463846FFF7EBFEB5E726
:10499000D8F81030B34208D01444211AC8F81C00CB
:1049A000A960BDE8F047FFF7F3BEBDE8F08700BFA0
:1049B000804B0020704B002038B501F007FA054A03
:1049C000D2E90845031B181945F10001C2E90801A5
:1049D00038BD00BF704B002000207047FEE700008C
:1049E000704700004FF0FF307047000002290CD0E4
:1049F000032904D00129074818BF00207047032A63
:104A000005D8054800EBC2007047044870470020F5
:104A1000704700BF386700082C230020EC660008B0
:104A200070B59AB00546084601A9144600F0C2F8D0
:104A300001A8FCF7FDFE431C5B00C5E90034002221
:104A4000237003236370C6B201AB02341046D1B2A7
:104A50008E4204F1020401D81AB070BD13F8011B94
:104A600004F8021C04F8010C0132F0E708B5302309
:104A700083F311880348FFF739FA002383F3118881
:104A800008BD00BFE04D002090F8443003F01F0245
:104A9000012A07D190F845200B2A03D10023C0E951
:104AA0000E3315E003F06003202B08D1B0F8483036
:104AB0002BB990F84520212A03D81F2A04D8FFF7E4
:104AC000F7B9222AEBD0FAE7034A82630722C263CE
:104AD00003640120704700BF2423002007B5052987
:104AE00017D8DFE801F0191603191920302383F3D2
:104AF0001188104A01900121FFF79AFA01980E4A95
:104B00000221FFF795FA0D48FFF7BCF9002383F364
:104B1000118803B05DF804FB302383F31188074844
:104B2000FFF786F9F2E7302383F311880348FFF794
:104B30009DF9EBE78C660008B0660008E04D0020A8
:104B400038B50C4D0C4C0D492A4604F10800FFF70E
:104B500067FF05F1CA0204F110000949FFF760FF81
:104B600005F5CA7204F118000649BDE83840FFF7A0
:104B700057BF00BFA85200202C2300206C660008FD
:104B8000766600088166000870B5044608460D4642
:104B9000FCF74EFEC6B22046013403780BB9184626
:104BA00070BD32462946FCF72FFE0028F3D10120C4
:104BB000F6E700002DE9F04705460C46FCF738FE05
:104BC0002B49C6B22846FFF7DFFF08B10B36F6B215
:104BD00028492846FFF7D8FF08B11036F6B2632EF1
:104BE0000BD8DFF88C80DFF88C90234FDFF894A08F
:104BF0002E7846B92670BDE8F08729462046BDE8E4
:104C0000F04701F089BC252E2ED1072241462846C7
:104C1000FCF7FAFD70B9194B224603F1100153F865
:104C2000040B42F8040B8B42F9D11B881380073523
:104C30001234DDE7082249462846FCF7E5FD98B91D
:104C40000F4BA21C197809090232C95D02F8041C35
:104C500013F8011B01F00F015345C95D02F8031C55
:104C6000F0D118340835C3E704F8016B0135BFE70C
:104C7000586700088166000860670008366500080C
:104C8000107AFF1F1C7AFF1FBFF34F8F024AD368B1
:104C9000DB03FCD4704700BF003C024008B5094B61
:104CA0001B7873B9FFF7F0FF074B1A69002ABFBFE3
:104CB000064A5A6002F188325A601A6822F4806209
:104CC0001A6008BD06550020003C024023016745DC
:104CD00008B50B4B1B7893B9FFF7D6FF094B1A6940
:104CE00042F000421A611A6842F480521A601A684F
:104CF00022F480521A601A6842F480621A6008BD79
:104D000006550020003C02400B28F0B516D80C4C8C
:104D10000C4923787BB90C4D0E460C234FF00062F2
:104D200055F8047B46F8042B013B13F0FF033A448B
:104D3000F6D10123237051F82000F0BD0020FCE7DC
:104D4000385500200855002074670008014B53F8BF
:104D500020007047746700080C2070470B2810B5BE
:104D6000044601D9002010BDFFF7CEFF064B53F8D3
:104D700024301844C21A0BB90120F4E7126801323A
:104D8000F0D1043BF6E700BF746700080B2810B5AC
:104D9000044621D8FFF778FFFFF780FF0F4AF3237F
:104DA000D360C300DBB243F4007343F0020313612A
:104DB000136943F480331361FFF766FFFFF7A4FF25
:104DC000074B53F8241000F03DF9FFF781FF204610
:104DD000BDE81040FFF7C2BF002010BD003C0240FC
:104DE00074670008F8B512F00103144642D1821826
:104DF000B2F1016F57D82D4B1B6813F0010352D04D
:104E00002B4DFFF74BFFF323EB60FFF73DFF40F225
:104E10000127032C15D824F001046618244C401AED
:104E200040F20117B142236900EB010524D123F0C0
:104E300001032361FFF74CFF0120F8BD043C04305F
:104E4000E7E78307E7D12B6923F440732B612B69D4
:104E50003B432B6151F8046B0660BFF34F8FFFF7A4
:104E600013FF03689E42E9D02B6923F001032B61F5
:104E7000FFF72EFF0020E0E723F44073236123694E
:104E80003B4323610B882B80BFF34F8FFFF7FCFE62
:104E90002D8831F8023BADB2AB42C3D0236923F079
:104EA00001032361E4E71846C7E700BF003802406A
:104EB000003C0240084908B50B7828B11BB9FFF740
:104EC000EDFE01230B7008BD002BFCD0BDE80840AF
:104ED0000870FFF7FDBE00BF0655002008B5064963
:104EE000064800F0B1F8BDE808404FF480314FF0BB
:104EF000805000F0A9B800BF00FF010000010020B1
:104F00000846114601F06CBA012001F069BA0000B0
:104F1000084601F083BA000038B5EFF311859DB95A
:104F2000EFF30584C4F30804302334B183F311880C
:104F3000FFF742FD85F3118838BD83F31188FFF731
:104F40003BFD84F3118838BDBDE83840FFF734BD20
:104F500038B5FFF7E1FF114C114AC00840EA417033
:104F6000A0FB025EC908A0FB040C1CEB050CA1FB16
:104F700004404FF000035B41A1FB02121CEB040C48
:104F800043EB000011EB0E0142F10002411842F127
:104F90000000090941EA007038BD00BFCFF753E3B4
:104FA000A59BC42010B50244064BD2B2904200D15A
:104FB00010BD441C00B253F8200041F8040BE0B2CD
:104FC000F4E700BF502800400F4B30B51C6F24049D
:104FD00007D41C6F44F400741C671C6F44F4004435
:104FE0001C670A4C236843F4807323600244084B17
:104FF000D2B2904200D130BD441C00B251F8045BE3
:1050000043F82050E0B2F4E700380240007000405E
:105010005028004007B5012201A90020FFF7C2FF78
:10502000019803B05DF804FB13B50446FFF7F2FFE7
:10503000A04205D0012201A900200194FFF7C4FF7E
:1050400002B010BD704700007047000070470000BC
:10505000074B45F255521A6002225A6040F6FF7221
:105060009A604CF6CC421A60024B01221A707047CB
:105070000030004040550020034B1B781BB1034B10
:105080004AF6AA221A6070474055002000300040BE
:10509000034B1A681AB9034AD2F874281A60704789
:1050A0003C55002000300240024B4FF08072C3F8A4
:1050B000742870470030024008B5FFF7E9FF024B43
:1050C0001868C0F3407008BD3C55002008B5FFF7D4
:1050D000DFFF024B1868C0F3007008BD3C5500208C
:1050E00070470000FEE700000A4B0B480B4A904255
:1050F0000BD30B4BDA1C121AC11E22F003028B4297
:1051000038BF00220021FCF79BBB53F8041B40F87A
:10511000041BECE790690008445600204456002028
:105120004456002070B5D0E915439E6800224FF028
:10513000FF3504EB42135101D3F800090028BEBF2C
:10514000D3F8000940F08040C3F80009D3F8000B01
:105150000028BEBFD3F8000B40F08040C3F8000B1E
:10516000013263189642C3F80859C3F8085BE0D2CD
:105170004FF00113C4F81C3870BD0000890141F0E4
:105180002001016103699B06FCD41220FFF76CBA71
:1051900010B5054C2046FEF72BFF4FF0A04363658A
:1051A000024BA36510BD00BF44550020C86700082E
:1051B00070B50378012B054650D12A4B446D9842B7
:1051C0001BD1294B5A6B42F080025A635A6D42F050
:1051D00080025A655A6D5A6942F080025A615A69D2
:1051E00022F080025A610E2143205B69FEF74AFDDE
:1051F0001E4BE3601E4BC4F800380023C4F8003E89
:10520000C02323606E6D4FF40413A3633369002B36
:10521000FCDA012333610C20FFF726FA3369DB0740
:10522000FCD41220FFF720FA3369002BFCDA0026A9
:10523000A6602846FFF776FF6B68C4F81068DB6845
:10524000C4F81468C4F81C684BB90A4BA3614FF04A
:10525000FF336361A36843F00103A36070BD064B95
:10526000F4E700BF445500200038024040140040DD
:1052700003002002003C30C0083C30C0F8B5446D4B
:10528000054600212046FFF779FFA96D00234FF066
:1052900001128F68C4F834384FF00066C4F81C2837
:1052A0004FF0FF3004EB431201339F42C2F8006914
:1052B000C2F8006BC2F80809C2F8080BF2D20B68FA
:1052C0006A6DEB65636210231361166916F01006B0
:1052D000FBD11220FFF7C8F9D4F8003823F4FE639D
:1052E000C4F80038A36943F4402343F01003A361DA
:1052F0000923C4F81038C4F814380A4BEB604FF097
:10530000C043C4F8103B084BC4F8003BC4F8106914
:10531000C4F80039EB6D03F1100243F48013EA6521
:10532000A362F8BDA467000840800010426D90F8A9
:105330004E10D2F8003823F4FE6343EA0113C2F89A
:10534000003870472DE9F84300EB8103456DDA68BA
:10535000166806F00306731E022B05EB41130C467C
:1053600080460FFA81F94FEA41104FF00001C3F86F
:10537000101B4FF0010104F1100398BFB60401FAAD
:1053800003F391698EBF334E06F1805606F5004651
:1053900000293AD0578A04F15801490137436F5028
:1053A000D5F81C180B43C5F81C382B180021C3F87E
:1053B000101953690127611EA7409BB3138A928B72
:1053C0009B08012A88BF5343D8F85C20981842EA0A
:1053D000034301F1400205EB8202C8F85C0021465C
:1053E00053602846FFF7CAFE08EB8900C3681B8A92
:1053F00043EA8453483464011E432E51D5F81C38C7
:105400001F43C5F81C78BDE8F88305EB4917D7F8AA
:10541000001B21F40041C7F8001BD5F81C1821EA35
:105420000303C0E704F13F0305EB83030A4A5A6014
:1054300028462146FFF7A2FE05EB4910D0F80039B7
:1054400023F40043C0F80039D5F81C3823EA0707D5
:10545000D7E700BF0080001000040002826D1268D0
:10546000C265FFF75FBE00005831436D49015B58CC
:1054700013F4004004D013F4001F0CBF02200120DD
:10548000704700004831436D49015B5813F40040F8
:1054900004D013F4001F0CBF02200120704700004D
:1054A00000EB8101CB68196A0B6813604B6853608D
:1054B0007047000000EB810330B5DD68AA6913680E
:1054C000D36019B9402B84BF402313606B8A1468E2
:1054D000426D1C44013CB4FBF3F46343033323F0FB
:1054E000030302EB411043EAC44343F0C043C0F856
:1054F000103B2B6803F00303012B09B20ED1D2F845
:10550000083802EB411013F4807FD0F8003B14BF41
:1055100043F0805343F00053C0F8003B02EB4112CC
:10552000D2F8003B43F00443C2F8003B30BD00001A
:105530002DE9F041244D6E6D06EB40130446D3F87F
:10554000087BC3F8087B38070AD5D6F81438190742
:1055500006D505EB84032146DB6828465B6898473F
:10556000FA071FD5D6F81438DB071BD505EB8403E3
:10557000D968CCB98B69488A5A68B2FBF0F600FB4F
:1055800016228AB91868DA6890420DD2121AC3E955
:105590000024302383F311880B482146FFF78AFF4C
:1055A00084F31188BDE8F081012303FA04F26B89CA
:1055B00023EA02036B81CB68002BF3D0214602481B
:1055C000BDE8F041184700BF4455002000EB8103BF
:1055D00070B5DD68436D6C692668E6604A0156BBAC
:1055E0001A444FF40020C2F810092A6802F003029E
:1055F000012A0AB20ED1D3F8080803EB421410F4C2
:10560000807FD4F8000914BF40F0805040F0005073
:10561000C4F8000903EB4212D2F8000940F004403C
:10562000C2F80009D3F83408012202FA01F101435B
:10563000C3F8341870BD19B9402E84BF40202060D3
:1056400020682E8A8419013CB4FBF6F440EAC44079
:1056500040F000501A44C6E72DE9F8433B4D6E6D0B
:1056600006EB40130446D3F80889C3F8088918F0FC
:10567000010F4FEA40171AD0D6F81038DB0716D5BD
:1056800005EB8003D9684B691868DA68904230D21C
:10569000121A4FF000091A60C3F80490302383F304
:1056A000118821462846FFF791FF89F3118818F0E9
:1056B000800F1CD0D6F834380126A640334216D0CD
:1056C00005EB84036D6DD3F80CC0DCF814200134B5
:1056D000E4B2D2F800E005EB04342F445168714580
:1056E00015D3D5F8343823EA0606C5F83468BDE882
:1056F000F883012303FA04F22B8923EA02032B81A6
:105700008B68002BD3D0214628469847CFE7BCF8BA
:105710001000AEEB0103834228BF0346D7F81809F7
:1057200080B2B3EB800FE2D89068A0F1040959F879
:10573000048FC4F80080A0EB09089844B8F1040F66
:10574000F5D818440B4490605360C7E744550020D7
:105750002DE9F74FA24C656D6E69AB691E4016F4DA
:1057600080586E6107D02046FEF7AAFC03B0BDE862
:10577000F04FFEF75DBA002E12DAD5F8003E9848D9
:105780009B071EBFD5F8003E23F00303C5F8003E7B
:10579000D5F8043823F00103C5F80438FEF7BAFC45
:1057A000370505D58E48FFF7BDFC8D48FEF7A0FCF8
:1057B000B0040CD5D5F8083813F0060FEB6823F4C5
:1057C00070530CBF43F4105343F4A053EB60310704
:1057D0001BD56368DB681BB9AB6923F00803AB61B9
:1057E0002378052B0CD1D5F8003E7D489A071EBFC3
:1057F000D5F8003E23F00303C5F8003EFEF78AFC0F
:105800006368DB680BB176489847F30274D4B7023B
:1058100027D5D4F85490DFF8C8B100274FF0010A1B
:1058200009EB4712D2F8003B03F44023B3F5802F75
:1058300011D1D2F8003B002B0DDA62890AFA07F386
:1058400022EA0303638104EB8703DB68DB6813B19F
:10585000394658469847A36D01379B68FFB29F426F
:10586000DED9F00617D5676D3A6AC2F30A1002F066
:105870000F0302F4F012B2F5802F00F08580B2F52C
:10588000402F08D104EB83030022DB681B6A07F575
:10589000805790426AD13003D5F8184813D5E103F8
:1058A00002D50020FFF744FEA20302D50120FFF736
:1058B0003FFE630302D50220FFF73AFE270302D51D
:1058C0000320FFF735FE75037FF550AFE00702D5E3
:1058D0000020FFF7C1FEA10702D50120FFF7BCFEA3
:1058E000620702D50220FFF7B7FE23077FF53EAF20
:1058F0000320FFF7B1FE39E7636DDFF8E4A0019301
:1059000000274FF00109A36D9B685FFA87FB9B4559
:105910003FF67DAF019B03EB4B13D3F8001901F465
:105920004021B1F5802F1FD1D3F8001900291BDACF
:10593000D3F8001941F09041C3F80019D3F80019C9
:105940000029FBDB5946606DFFF718FC218909FA35
:105950000BF321EA0303238104EB8B03DB689B68D1
:1059600013B15946504698470137CCE7910708BF15
:10597000D7F80080072A98BF03F8018B02F10102D3
:1059800098BF4FEA182884E7023304EB830207F537
:1059900080575268D2F818C0DCF80820DCE9001CF7
:1059A000A1EB0C0C002188420AD104EB830463684C
:1059B0009B699A6802449A605A6802445A606AE78E
:1059C00011F0030F08BFD7F800808C4588BF02F89C
:1059D000018B01F1010188BF4FEA1828E3E700BFFE
:1059E00044550020436D03EB4111D1F8003B43F4D3
:1059F0000013C1F8003B7047436D03EB4111D1F830
:105A0000003943F40013C1F800397047436D03EBCC
:105A10004111D1F8003B23F40013C1F8003B70475B
:105A2000436D03EB4111D1F8003923F40013C1F8A1
:105A30000039704730B5039C0172043304FB032521
:105A4000C0E90653049B03630021059BC160C0E9C4
:105A50000000C0E90422C0E90842C0E90A1143631A
:105A600030BD0000416A0022C0E90411C0E90A22E9
:105A7000C2606FF00101FEF767BE0000D0E904329A
:105A8000934201D1C2680AB9181D704700207047BF
:105A900003691960C2680132C260C2691344826935
:105AA0000361934224BF436A03610021FEF740BEB5
:105AB00038B504460D46E3683BB16269131D1268B0
:105AC000A3621344E362002007E0237A33B9294636
:105AD0002046FEF71DFE0028EDDA38BD6FF001000C
:105AE000FBE70000C368C269013BC360436913441C
:105AF00082694361934224BF436A43610023836206
:105B0000036B03B11847704770B53023044683F325
:105B10001188866A3EB9FFF7CBFF054618B186F3B8
:105B20001188284670BDA36AE26A13F8015BA3627C
:105B3000934202D32046FFF7D5FF002383F3118859
:105B4000EFE700002DE9F84F04460E461746984649
:105B50004FF0300989F311880025AA46D4F828B0FF
:105B6000BBF1000F09D141462046FFF7A1FF20B14C
:105B70008BF311882846BDE8F88FD4E90A12A7EB09
:105B8000050B521A934528BF9346BBF1400F1BD912
:105B9000334601F1400251F8040B43F8040B9142E3
:105BA000F9D1A36A40334036A3624035D4E90A23D1
:105BB0009A4202D32046FFF795FF8AF31188BD422F
:105BC000D8D289F31188C9E730465A46FBF712FE4E
:105BD000A36A5B445E44A3625D44E7E710B5029CA0
:105BE0000172043303FB0421C0E906130023C0E95A
:105BF0000A33039B0363049BC460C0E90000C0E94F
:105C00000422C0E90842436310BD0000026AC2607A
:105C1000426AC0E904220022C0E90A226FF00101B1
:105C2000FEF792BDD0E904239A4201D1C26822B99D
:105C3000184650F8043B0B60704700231846FAE7FB
:105C4000C368C2690133C360436913448269436115
:105C5000934224BF436A43610021FEF769BD0000FF
:105C600038B504460D46E3683BB123691A1DA262AC
:105C7000E2691344E362002007E0237A33B929463E
:105C80002046FEF745FD0028EDDA38BD6FF0010033
:105C9000FBE7000003691960C268013AC260C2698B
:105CA000134482690361934224BF436A0361002362
:105CB0008362036B03B118477047000070B530234F
:105CC0000D460446114683F31188866A2EB9FFF704
:105CD000C7FF10B186F3118870BDA36A1D70A36A57
:105CE000E26A01339342A36204D3E1692046043996
:105CF000FFF7D0FF002080F31188EDE72DE9F84F82
:105D000004460D46904699464FF0300A8AF31188B2
:105D10000026B346A76A4FB949462046FFF7A0FFC1
:105D200020B187F311883046BDE8F88FD4E90A071F
:105D30003A1AA8EB0607974228BF1746402F1BD9EF
:105D400005F1400355F8042B40F8042B9D42F9D18E
:105D5000A36A4033A3624036D4E90A239A4204D3AB
:105D6000E16920460439FFF795FF8BF3118846451A
:105D7000D9D28AF31188CDE729463A46FBF73AFD96
:105D8000A36A3B443D44A3623E44E5E7D0E90423D3
:105D90009A4217D1C3689BB1836A8BB1043B9B1AAB
:105DA0000ED01360C368013BC360C3691A448369A2
:105DB00002619A4224BF436A036100238362012384
:105DC000184670470023FBE700F0D2B84FF080433D
:105DD000586A70474FF08043002258631A610222CC
:105DE000DA6070474FF080430022DA6070470000AD
:105DF0004FF0804358637047FEE7000070B51B4BBF
:105E000001630025044686B0586085620E46FDF7A2
:105E1000EBFE04F11003C4E904334FF0FF33C4E98F
:105E20000635C4E90044A560E562FFF7CFFF2B46C5
:105E30000246C4E9082304F134010D4A2565802394
:105E40002046FEF71BFC0123E0600A4A037500921E
:105E500072680192B268CDE90223074B6846CDE92A
:105E60000435FEF733FC06B070BD00BFD84D0020EE
:105E7000D4670008D9670008F95D0008024AD36AB0
:105E80001843D062704700BF704B00204B684360DE
:105E90008B688360CB68C3600B6943614B690362A5
:105EA0008B6943620B6803607047000008B5264B9E
:105EB00026481A6940F2FF110A431A611A6922F44E
:105EC000FF7222F001021A611A691A6B0A431A63FF
:105ED0001A6D0A431A651E4A1B6D1146FFF7D6FF5D
:105EE00002F11C0100F58060FFF7D0FF02F13801DC
:105EF00000F58060FFF7CAFF02F1540100F58060F1
:105F0000FFF7C4FF02F1700100F58060FFF7BEFFEC
:105F100002F18C0100F58060FFF7B8FF02F1A801E3
:105F200000F58060FFF7B2FF02F1C40100F5806068
:105F3000FFF7ACFF02F1E00100F58060FFF7A6FF7C
:105F4000BDE8084000F090B8003802400000024070
:105F5000E067000808B500F0FBF9FEF75DFBFFF70E
:105F600097F8BDE80840FEF7EBBD00007047000061
:105F70000F4B1A6C42F001021A641A6E42F00102D1
:105F80001A660C4A1B6E936843F0010393604FF04E
:105F9000804353229A624FF0FF32DA6200229A6104
:105FA0005A63DA605A6001225A611A60704700BF72
:105FB00000380240002004E04FF0804208B511692B
:105FC000D3680B40D9B2C9439B07116107D5302371
:105FD00083F31188FEF746FB002383F3118808BD85
:105FE0001F4B1A696FEAC2526FEAD2521A611A69DC
:105FF000C2F308021A614FF0FF301A695A695861FA
:1060000000215A6959615A691A6A62F080521A620B
:106010001A6A02F080521A621A6A5A6A58625A6AF6
:1060200059625A6A1A6C42F080521A641A6E42F02F
:1060300080521A661A6E0B4A106840F48070106025
:10604000186F00F44070B0F5007F1EBF4FF4803031
:1060500018671967536823F40073536000F054B94C
:106060000038024000700040334B4FF080521A64F9
:10607000324A4FF4404111601A6842F001021A603E
:106080001A689107FCD59A6822F003029A602A4B9D
:106090009A6812F00C02FBD1196801F0F90119603D
:1060A0009A601A6842F480321A601A689203FCD52A
:1060B0005A6F42F001025A671F4B5A6F9007FCD586
:1060C0001F4A5A601A6842F080721A601B4A53686D
:1060D0005904FCD5184B1A689201FCD5194A9A60EC
:1060E000194B1A68194B9A42194B21D1194A116858
:1060F000194A91421CD140F205121A60144A1368E1
:1061000003F00F03052BFAD10B4B9A6842F0020201
:106110009A609A6802F00C02082AFAD15A6C42F48A
:1061200080425A645A6E42F480425A665B6E7047EF
:1061300040F20572E1E700BF003802400070004005
:106140000854400700948838002004E011640020BF
:10615000003C024000ED00E041C20F41074A08B593
:10616000536903F00103536123B1054A13680BB16E
:1061700050689847BDE80840FDF75ABD003C014013
:10618000BC550020074A08B5536903F00203536168
:1061900023B1054A93680BB1D0689847BDE8084021
:1061A000FDF746BD003C0140BC550020074A08B53C
:1061B000536903F00403536123B1054A13690BB11A
:1061C00050699847BDE80840FDF732BD003C0140EA
:1061D000BC550020074A08B5536903F00803536112
:1061E00023B1054A93690BB1D0699847BDE80840CF
:1061F000FDF71EBD003C0140BC550020074A08B514
:10620000536903F01003536123B1054A136A0BB1BC
:10621000506A9847BDE80840FDF70ABD003C0140C0
:10622000BC550020164B10B55C6904F478725A61B5
:10623000A30604D5134A936A0BB1D06A9847600647
:1062400004D5104A136B0BB1506B9847210604D547
:106250000C4A936B0BB1D06B9847E20504D5094A01
:10626000136C0BB1506C9847A30504D5054A936C89
:106270000BB1D06C9847BDE81040FDF7D9BC00BF0A
:10628000003C0140BC550020194B10B55C6904F47A
:106290007C425A61620504D5164A136D0BB1506DEC
:1062A0009847230504D5134A936D0BB1D06D9847D9
:1062B000E00404D50F4A136E0BB1506E9847A10449
:1062C00004D50C4A936E0BB1D06E9847620404D586
:1062D000084A136F0BB1506F9847230404D5054A41
:1062E000936F0BB1D06F9847BDE81040FDF7A0BC8D
:1062F000003C0140BC55002008B5FFF75DFEBDE83D
:106300000840FDF795BC0000062108B50846FDF7DA
:10631000B9FC06210720FDF7B5FC06210820FDF792
:10632000B1FC06210920FDF7ADFC06210A20FDF78E
:10633000A9FC06211720FDF7A5FC06212820FDF762
:10634000A1FCBDE8084007211C20FDF79BBC000014
:1063500008B5FFF745FE00F00BF8FDF747FEFDF727
:106360001FFDFFF703FEBDE80840FFF72DBD00004D
:106370000023054A19460133102BC2E9001102F12E
:106380000802F8D1704700BFBC5500200B460146FB
:10639000184600F02DB8000000F040B8012838BFC2
:1063A000012010B50446204600F030F830B900F066
:1063B00007F808B900F00CF88047F4E710BD0000BA
:1063C000024B1868BFF35B8F704700BF3C5600203C
:1063D00008B5062000F084F80120FEF7FFFA00005F
:1063E000024B0A4601461868FEF78ABD4C2300207E
:1063F00010B5054C13462CB10A4601460220AFF3F6
:10640000008010BD2046FCE700000000024B014662
:106410001868FEF779BD00BF4C230020024B0146EF
:106420001868FEF775BD00BF4C23002010B5013978
:106430000244904201D1002005E0037811F8014F99
:10644000A34201D0181B10BD0130F2E72DE9F04145
:10645000A3B1C91A17780144044603F1FF3C8C42EA
:10646000204601D9002009E00578BD4204F101046D
:10647000F5D10CEB0405D618A54201D1BDE8F08199
:1064800015F8018D16F801EDF045F5D0E7E70000AD
:106490001F2938B504460D4604D9162303604FF072
:1064A000FF3038BD426C12B152F821304BB9204652
:1064B00000F030F82A4601462046BDE8384000F09A
:1064C00017B8012B0AD0591C03D1162303600120F1
:1064D000E7E7002442F82540284698470020E0E7F7
:1064E000024B01461868FFF7D3BF00BF4C230020C2
:1064F00038B5074D00230446084611462B60FEF7C9
:1065000071FA431C02D12B6803B1236038BD00BF70
:1065100040560020FEF760BA034611F8012B03F83D
:10652000012B002AF9D170476F72672E6172647572
:1065300070696C6F742E663430352D4D6174656BE7
:1065400041697273706565640000000053544D33F7
:1065500032463F3F3F0053544D333246343078008B
:1065600053544D3332463432780053544D3332460F
:106570003434365858000000012033000010410028
:1065800001105A00031059000710310000000000EC
:106590004C6500081304000056650008190400004B
:1065A00060650008210400006A65000840A2E4F16B
:1065B000646891060041A3E5F26569920700000056
:1065C0004261642043414E496661636520696E649F
:1065D00065782E0080000000008000000000800030
:1065E0000000000000000000FD2000081D29000838
:1065F000792800083D2100084921000849230008A6
:106600000D2100081D210008112100081921000892
:10661000152100086D22000821210008ED2B00083B
:106620003121000841220008000000001D3D000843
:10663000093D0008453D0008313D00083D3D00088A
:10664000293D0008153D0008013D0008513D0008A6
:1066500000000000010000000000000063300000A6
:106660005C660008C84B0020D84D0020417264755C
:1066700050696C6F740025424F415244252D424CA5
:10668000002553455249414C2500000002000000FE
:1066900000000000393F0008A53F0008400040000E
:1066A0007852002088520020020000000000000004
:1066B0000300000000000000E93F000800000000A7
:1066C00010000000985200200000000001000000AF
:1066D000000000004455002001010200DD4A0008CE
:1066E000ED490008894A00086D4A0008430000008F
:1066F000F466000809024300020100C032090400E8
:10670000000102020100052400100105240100011E
:10671000042402020524060001070582030800FF85
:1067200009040100020A0000000705010240000000
:1067300007058102400000001200000040670008C9
:10674000120110010200004009124157000201022B
:10675000030100000403090425424F41524425006F
:106760003031323334353637383941424344454687
:106770000000000000400000004000000040000059
:1067800000400000000001000000020000000200C4
:1067900000000200000002000000020000000200F1
:1067A00000000200000000002D410008E543000841
:1067B0009144000840004000A4550020A45500204A
:1067C00001000000B45500208000000040010000DE
:1067D000030000006D61696E0069646C6500000073
:1067E000AA01A81200000000AAAAAAAA5501140032
:1067F000FFBF00008877000070A70A0000000A01B0
:1068000000000000AAAAAAAA00000001FFFF0000E1
:1068100000000000990000000000A0160000000029
:10682000AAAAAAA600005011FFDF00000000000085
:10683000007708002000000000000000AAAAAAAA11
:1068400010000000FFFF0000000800000000000032
:106850000000000000000000AAAAAAAA0000000090
:10686000FFFF00000000000000000000000000002A
:1068700000000000AAAAAAAA00000000FFFF000072
:106880000000000000000000000000000000000008
:10689000AAAAAAAA00000000FFFF00000000000052
:1068A0000000000000000000000000000A000000DE
:1068B00000000000030000000000000000000000D5
:1068C00000000000000000000000000000000000C8
:1068D00000000000000000000000000000000000B8
:1068E000F60300000000000000000F0000000000A0
:1068F00040420F00FE2A0100D2040000FF00960073
:1069000000000008009600000000080004000000DD
:1069100054670008000000000000000000000000B4
:1069200000000000000000000000000050230020D4
:106930000000000000000000000000000000000057
:106940000000000000000000000000000000000047
:106950000000000000000000000000000000000037
:106960000000000000000000000000000000000027
:106970000000000000000000000000000000000017
:106980000000000000000000000000000000000007
:00000001FF
